:0E741A00C29CD2A08F993099FDC2A0C29922C7
:105A4200126608306D2053B1F8C26D1272DB127407
:105A520040127175126D90126520126815126FA1B5
:105A620012580B12729B306C21B2A4C26C121C7AB7
:105A7200125D901272251271B21271CF125CC54082
:105A8200031250EC1272C6124561126FCE1271EC03
:105A92001263951247BB124E48900206E524F0A30A
:0E5AA200E525F0A3E522F0A3E523F08096228F
:106B20009005367401F07E027F3C7B40E4FD1270DC
:106B3000257E027F0A7B14E4127025900224740AD9
:106B4000F0A374ABF0A3740AF0A374ABF0C22CC230
:106B50002D9003FF7402F0D22ED27B90027C7450F1
:026B6000F02221
:1050EC007FFE7E0112704F501F7B007A02E4FDFCA4
:1050FC00FFFE125F107FFE7E0312704F402CE4FD0A
:10510C00FF7E021252C080227FFE7E0312704F502F
:10511C00167B007A02E4FDFCFF7E02125F10E4FDB8
:10512C00FFFE1252C08003D26E22900000E0F520E8
:10513C00A3E0F521900238E520F0A3E521F09000E2
:10514C001A12275190022C1227B7900022E0FFA3CD
:10515C00E0900236CFF0A3EFF0E52154072403F5DD
:10516C001364056005E513B40A04E4F51422E51391
:10517C0064046005E513B409047514012275140266
:01518C002200
:10719400C2AFD2ACC086758640C28FD086D2AD4312
:0E71A400BA6043E840E4F5D843A908D2AF2210
:106FFA007580F075E18F75E9C075908075E27F75CF
:10700A00EA8075A04675E3BB75EB4675B01875E462
:0B701A00E675EC184380C043E98022BB
:10660800E4FF127133126FFA1250EC126B207D0501
:106618007C007F44126F71125DF112726E7D647F8F
:10662800A07E0F12570D1255851254FE4002D25A01
:10663800126CDE30071212578E4002D2397E047F68
:0C664800971253E54002D27812719422A0
:10102E00EFB4200E206303306619E4FF127133D241
:10103E006522EFB4400D206303306607E4FF1271A2
:04104E0033D2652212
:10710F00D26B90049FE004F0C3940A4004E4F0D2E1
:10711F006D90049EE004F0C394C84004E4F0D26C78
:04712F0012504A228E
:106C2300D3EF9450EE940040037F0522D3EF943CBE
:106C3300EE940040037F0422D3EF9428EE940040A7
:106C4300037F0322D3EF9414EE940040037F0222C8
:0F6C5300D3EF9400EE940040037F01227F0022D4
:1072EF0030710F90053EE004F0C394644004E4F065
:0372FF00C2712237
:105FCC00302A1490053CE004F0C3940A400BE4F032
:105FDC00A2B5B392B58002C2B530720D90053DE00A
:105FEC0004F0C394054002E4F030712C900234E0CC
:105FFC00FEA3E0FF126C23EF6401601CEFB40204FB
:10600C00D2A18014EFB40306D2A1D2A2800AEFB4BD
:0B601C000406D2A1D2A2D2A31272EFA0
:016027002256
:105C5F00C22CC22DC22E302B569003FFE0701804B9
:105C6F00F0D22D900089E0FEA3E0FF90008CE0FDC4
:105C7F0012570D43B701229003FFE0B401167402CF
:105C8F00F0D22E900089E0FEA3E0FF7D6412570D45
:105C9F0043B70122E49003FFF0D22C900089E0FE7D
:105CAF00A3E0FF90008BE0FD12570D43B70122C216
:065CBF002CC22DC22E22B2
:106F4100307A2CC27AE50824FE600F24F160161411
:106F5100601024117019125C5F22D271E490053E19
:106F6100F022D26322B272307203C28322D2832210
:106BA30030653CC265306624E4FF127133D2AFC254
:106BB30066E49005E8F07F01126936D2ACD2ADD21B
:106BC300CE7F701272571273C012734EE49005E8B1
:106BD300F0A3F09003F7F09003F8F09003F9F0229C
:1073E60053B1F8C2AFD283E4FF1272B112709D801E
:0273F600EF2284
:106E0500D283C2721273611273D37F701273F8C288
:106E1500CE53B77E302904D2A58002C2A57F0112C8
:106E25006936C2AFC2ACC2ADE4F5D87F801271330A
:066E3500D2AF12743422FA
:1053570030640E204306204403304505C264D263FF
:105367002230161490002AE0FF9005E9E004F0C30C
:105377009F406AEFF0D2632220715B202A50202BD6
:105387004D30191490002AE0FF9005E9E004F0C3BE
:105397009F404AEFF0D26322E49005E9F0A212722F
:1053A700107218721A721172137219721B721C72B0
:1053B700157272401390002AE0FF9005E8E004F0B0
:1053C7009F401AEFF0D26622E49005E8F022E490BD
:0E53D70005E8F0A3F022E49005E8F0A3F02230
:106BE300206626206323C2AFA279727A726F726520
:106BF300724C726D726C400D9005EAE06412600590
:106C0300D2AF127428D2AF801330630AD26F124707
:106C1300BB1273E68006306603126E05126BA32265
:10685E00000000300062007400000089008E009974
:10686E0000A200AA00BB00BF00FE00000000000056
:10687E00000000000020005000820094000000A9DB
:10688E0000AE00B900C200CA00DB00DF011E00002E
:08689E000000000000000000F2
:10728500900402E07008C29C75995AD2A022C29C53
:067295007599FFD2A02252
:085881009002B8EEF0A3EFF075
:105889007B017A047900900402E02403FD12720975
:10589900900402E02403F582E43404F583E06F7098
:1058A90043FF900402E0FEEFC39E502953B1F87400
:1058B900032FF582E43404F583E0FE9002B8E0FC9E
:1058C900A3E0F5828C83EEF09002B8E475F0011242
:1058D900257B0F80CDD270E49005F5F0C29C7599B7
:0B58E9005AD2A022C29C7599FFD2A0E9
:0158F4002291
:105D2B00900402E0D3948C4002E4F0E4FD90040272
:105D3B00E0FCEDC39C501D53B1F88F828E83E0FBCA
:105D4B0074032DF582E43404F583EBF00FBF0001EF
:105D5B000E0D80D97B017A047900EC2403FD1272BD
:105D6B0009900402E02403F582E43404F583EFF098
:105D7B00C29C9003FAE02400F582E43404F583E03E
:045D8B00F599D2A014
:015D8F0022F1
:1067CC007B017A047900900402E02403FD12720923
:1067DC00900402E02403F582E43404F583E0B50769
:1067EC0020900404E0FFB441089005EA7412F08094
:1067FC0006EFB40502D264C243C29C75995AD2A06A
:09680C0022C29C7599FFD2A02262
:106D1A007B017A047900900402E02403FD127209CF
:106D2A00900402E02403F582E43404F583E0B50715
:106D3A0012900403E09003F2F0C243C29C75995A80
:0B6D4A00D2A022C29C7599FFD2A022AB
:103B8800900401E0FF12280D3BDC013BDC023BDC2A
:103B9800033BDC043BDC053BDC063BDC073BDC0889
:103BA8003BDC093BDC0A3BED0B3BFD0C3C050D3CCB
:103BB8000D0E3C150F3BF5103C1D113C25123C2DFC
:103BC800133C35143C3D153C45163C4D173C5518E7
:103BD80000003C5DEF25E02408F582E43402AF8262
:103BE800FE125D2B227E027F1E125D2B227E027F3B
:103BF80020125D2B227E027F24125D2B227E027F03
:103C080026125D2B227E027F28125D2B227E027FE8
:103C18002A125D2B227E027F2C125D2B227E027FD0
:103C280030125D2B227E027F34125D2B227E027FB2
:103C380036125D2B227E027F06125D2B227E027FCA
:103C480008125D2B227E027F38125D2B227E027FB6
:103C58003A125D2B22900402E0C394804009D23AC4
:103C68009003E27401F022900401E0B4781090030C
:103C7800F2E0B40C09D23A9003EF7401F0229004F8
:103C880001E0B478229003F2E025E0245EF582E4B6
:103C98003468F583E493FE740193FF9002B6EEF066
:103CA800A3EFF0125D2B22900401E0B47921900378
:103CB800F2E025E02482F582E43468F583E493FE9B
:0F3CC800740193FF9002B6EEF0A3EFF0125D2BA4
:013CD70022CA
:106243007B017A047900900402E02403FD127209B1
:10625300900402E02403F582E43404F583E06F70D4
:106263002F900403E0FEA3E0FDEEEDFF9005DFEECB
:10627300F0A3EFF04E7008C29C7599FFD2A022D212
:10628300799005DAE04401F0C29C75995AD2A022B4
:08629300C29C7599FFD2A02204
:1046F8007B017A047900900402E02403FD12720918
:10470800900402E02403F582E43404F583E06F604A
:10471800030247B3900404E0FFE4FCFDFE781012A6
:104728002732C004C005C006C007900403E0FFE4B8
:10473800FCFDFE7818122732D003D002D001D00039
:104748001226C9C004C005C006C007900405E0FFD2
:10475800E4FCFDFE7808122732D003D002D001D045
:10476800001226C9A804A905AA06AB07A3E0FFE41E
:10477800FCFDFE1226C99005D61227B79002A1E0CB
:104788007002A3E0600C9005D6122751EC4D4E4FF5
:104798007008C29C7599FFD2A022D2799005DAE000
:1047A8004410F0C29C75995AD2A022C29C7599FFF8
:0347B800D2A0226A
:106DCB007B017A047900900402E02403FD1272091E
:106DDB00900402E02403F582E43404F583E0B50764
:106DEB0011D2799005DAE04420F0C29C75995AD201
:0A6DFB00A022C29C7599FFD2A022CD
:10656E007B017A047900900402E02403FD12720983
:10657E00900402E02403F582E43404F583E06F70A6
:10658E0024D279900403E0FEA3E0FDEEEDFF90052A
:10659E00DBEEF0A3EFF09005DAE04404F0C29C7558
:0D65AE00995AD2A022C29C7599FFD2A0225A
:1065BB007B017A047900900402E02403FD12720936
:1065CB00900402E02403F582E43404F583E06F7059
:1065DB0024D279900403E0FEA3E0FDEEEDFF9005DD
:1065EB00DDEEF0A3EFF09005DAE04408F0C29C7505
:0D65FB00995AD2A022C29C7599FFD2A0220D
:10629B007B017A047900900402E02403FD12720959
:1062AB00900402E02403F582E43404F583E06F707C
:1062BB002FFF74032FF582E43404F583E0FE74E1C1
:1062CB002FF582E43405F583EEF00FEFB407E3D23C
:1062DB00799005DAE04480F0C29C75995AD2A022DD
:0762EB00C29C7599FFD2A0CF
:0162F2002289
:104EF400900401E012280D4F20184F24774F40787A
:104F04004F62794F2CA04F34A14F38A24F28A34FA2
:104F140030A44F3CAF4F84B000004F9E1267CC22A8
:104F2400126D1A221246F82212624322126DCB220B
:104F340012656E221265BB2212629B229003F2E07C
:104F440025E0245EF582E43468F583E493FE74017D
:104F540093FF9002B6EEF0A3EFF012588122900373
:104F6400F2E025E02482F582E43468F583E493FEDC
:104F7400740193FF9002B6EEF0A3EFF01258812271
:104F8400900403E0B4550CD23AD238C29C75995AB5
:0A4F9400D2A022C29C7599FFD2A0A2
:014F9E0022F0
:1038B700E49002B6F0A3F09003FAE0FFB4021A9086
:1038C7000401E064A56006E49003FAF022E49003A3
:1038D700FDF0A3F09003F3F022900402E0FD7C00DA
:1038E7002409FBEC33FA7E00C3EF9BEA6480F8748B
:1038F7008098505FED2407FDEC33FCD3EF9DEC641B
:1039070080F874809850189003FAE024FFF582E459
:103917003403F583E0FF9003FDEE8FF012257B90D3
:1039270003FAE0FFB40511900404E0640770030292
:103937003A1FE49003FAF022EF64066003023A1F8D
:10394700900405E064067003023A1F9003F3E04415
:1039570020F022E49003FAF0900402E0FD2408F539
:1039670082E43404F583E0FE74072DF582E4340421
:10397700F583E07C002400FFEC3EFE9003FDE06E43
:103987007003A3E06F60079003F3E04480F09003B7
:10399700F3E0FF6006900406F08007D24CE4900441
:1039A70006F0E4900402F0900405740BF090040311
:1039B700E0FFA3E0900403F0A3EFF07F029004027E
:1039C700E0FE2407FDE433FCEFC39DEC6480F8744C
:1039D7008098501874002FF582E43404F583E0FDD5
:1039E7009002B6E48DF012257B0F80D19002B6E0ED
:1039F700FCA3E0FF74072EF582E43404F583EFF0AF
:103A0700ECFF900402E02408F582E43404F583EF28
:083A1700F0C29C75995AD2A07F
:013A1F002284
:105229009003FAE02400F582E43404F583EFF0906A
:1052390003FAE004F0E0C3948C4002E4F09003FA2E
:10524900E064017027900400E0FF54FEB59A10EF66
:1052590020E006D246C2498013D249C246800D9049
:105269000400E0645A6005E49003FAF030460D90BA
:1052790003FAE064037030123B88802B3049259093
:105289000402E02403FFE433FE9003FAE0D39FEE27
:105299006480F8748098400F124EF4C249E4900378
:1052A900FAF080031238B7C243E49005E8F090059C
:0752B900E9F09003F7F02279
:104CE200900400E0B45A06A3E064A56003304C4887
:104CF200900402E02408FFE433FE9003FAE0C39F2D
:104D0200EE6480F87480984016D29CC2A0E4F0C28F
:104D120046900400F0A3F0A3F0A3F0D24380669083
:104D220003FAE004F0C29CE02400F582E43404F5C6
:104D320083E0F599D2A0804D9003FAE0FF601690CF
:104D42000402E02403FDE433FCC3EF9DEC6480F82D
:104D52007480984019D29CC2A0E49003FAF0C24633
:104D6200900400F0A3F0A3F0A3F0D24380179003C5
:104D7200FAE004F0C29CE02400F582E43404F583F6
:104D8200E0F599D2A0E49005E8F09005E9F09003EF
:034D9200F7F02215
:10729B009003F7E004F0C39404400AE4F09003FA7F
:0672AB00F0D29CC2A022FB
:10722500305C119002B1E004F0C39405400BD25AD2
:0A7235007405F022E49002B1F0228B
:0E4F9F009002C1EFF0A3EDF0A3EAF0A3EBF057
:104FAD00C254E4A3F0305A03025042A3F09002C25F
:104FBD00E0FF9002C6E0C39F507B9002C5E0FF0466
:104FCD00F0EFC39405503E9002C1E0FD7C009002CD
:104FDD00FA7401F0A3F09002C3E0FFA3E09002FC8D
:104FED00CFF0A3EFF0E4FB7F36123CD8925430544F
:104FFD0004801280C5E4F5C87F0112693612726E05
:10500D0012693680B59002C5E0C394054004802531
:10501D008015E49002C5F09002C1E004F09002C347
:10502D00E475F00112257B7F011269369002C6E00E
:0C503D0004F0024FBAA254B3925CA254DB
:015049002244
:0E5B89009002C4EFF0A3EDF0A3EAF0A3EBF05E
:105B9700C254E4A3F0205A4D9002C8E0FF04F0EF8E
:105BA700C3940550409002C4E0FD7C00A3E090023E
:105BB700F0F0A37401F09002C6E0FFA3E09002F2B8
:105BC700CFF0A3EFF0E4FB7F3612325B92543054F0
:105BD70004801280C3E4F5C87F0112693612726E21
:0C5BE70012693680B3A254B3925CA25441
:015BF300228F
:106CDE007A027BA37D02E4FF125B89502E9002A301
:106CEE00E07004A3E060249002A7E04480F07A02F2
:106CFE007BA77D017F04124F9F9002A7E0547FF087
:0C6D0E007A027BA77D017F04124F9F22B8
:10558500E49002A6F0A37450F0E4A3F0A374F8F03D
:10559500E4A3F0A3F0A37470F0A37401F0A3740363
:1055A500F0A374FFF0E4A3F03000199002A7E044E3
:1055B50008F09002ACE0FF9000BBE0540FFEEF4E08
:1055C5009002ACF030013E9002A7E04404F0900256
:1055D500ADE0FF9000BBE054F0FEEF4E9002ADF061
:1055E5009000BCE0FEA3E0FF7C007D32122833E48E
:1055F5007B257A01F9F8122637AD07AC06EC900247
:05560500AEF0A3EFF080
:01560A00227D
:1054FE00D2539002C07403F09002C0E0FF14F0EF9C
:10550E0060727A027BA67D0B7F03124F9F505C90D8
:10551E0002BF7403F09002BFE0FFD3940B504E7A9B
:10552E00027BBD7D02125B899002BFE0FF7E007B95
:10553E000124A3F9EE3402FA1224FBFD9002BDE021
:10554E00B5051374A42FF9EE3402FA1224FBFF9062
:10555E0002BEE06F600C9002BFE064076004C253AD
:10556E00800B9002BFE02402F080AAC25330538811
:06557E0080028084A253AC
:015584002204
:106CA1007A027BA37D02E4FF125B89502F9002A43C
:106CB100E0FF30E102D259EF30E002D25B9002A353
:106CC100E0FF30E307206804D215D26AEF30E20218
:0D6CD100D2149002A4E030E2031254FE221F
:10723F007A027BBA7D027F02125B89500A9002BAF2
:07724F00E09002A5F0F52616
:017256002215
:105D90009002BC7403F09002BCE0FFD3940B50500F
:105DA0007A027BBA7D02125B899002BCE0FF7E0022
:105DB0007B0124A3F9EE3402FA1224FBFD9002BA0F
:105DC000E0B5051374A42FF9EE3402FA1224FBFF98
:105DD0009002BBE06F60109002BCE06407600812A4
:105DE00054FE400CD263229002BCE02402F080A654
:015DF0002290
:10709D009002B07433F07A027BB07D017F0D124FF8
:1070AD009F50129002A7E04420F07A027BA77D0149
:0670BD007F04124F9F2228
:1072B1009002A8E054FCF04FF07A027BA87D017F98
:0572C10005124F9F22A1
:107302009002A7E04401F07A027BA77D017F04127C
:037312004F9F2268
:107315009002A7E054FEF07A027BA77D017F04125C
:037325004F9F2255
:107328009002A7E04402F07A027BA77D017F041255
:037338004F9F2242
:10733B009002A7E054FDF07A027BA77D017F041237
:03734B004F9F222F
:106C62009002BCEEF0A3EFF09002BCE0FEA3E0784D
:106C720005CEC313CE13D8F99002AAF07A027BAAEA
:106C82007D017F07124F9F50159002BCE0A3E09058
:0F6C920002ABF07A027BAB7D017F08124F9F228D
:10734E009002A7E04410F07A027BA77D017F041221
:03735E004F9F221C
:107361009002A7E054EFF07A027BA77D017F04121F
:037371004F9F2209
:107374009002A9E044F8F07A027BA97D017F06120D
:037384004F9F22F6
:107387009002A9E05407F07A027BA97D017F0612DB
:037397004F9F22E3
:10739A009002A9E044E0F07A027BA97D017F0612FF
:0373AA004F9F22D0
:1073AD009002A9E0541FF07A027BA97D017F06129D
:0373BD004F9F22BD
:1073C0009002A9E04408F07A027BA97D017F0612B1
:0373D0004F9F22AA
:1073D3009002A9E054F7F07A027BA97D017F06129F
:0373E3004F9F2297
:1073F8009002A6E04FF07A027BA67D017F03124F30
:027408009F22C1
:107257009002A6E0FEEFF4FFEE5FF07A027BA67DD8
:07726700017F03124F9F227B
:103E1F00305E03023F62305F03023F622003030202
:103E2F003F62E490053AF0A3F0C3900063E095126F
:103E3F00900062E09511500330181ED3900065E09A
:103E4F009512900064E09511400320180C20100982
:103E5F00201206201103301308C260E4900539F0D8
:103E6F0022C39000A3E095129000A2E095114003A9
:103E7F00023F5BC3E5129510FFE511950FFED3903E
:103E8F0000A5E09F9000A4E09E4003023F5B9000DE
:103E9F00A6E0FEA3E0FFEE3395E0FDFC90022012BA
:103EAF00276AC31226E45003023F5B206006900589
:103EBF0039E004F09000A8E075F00AA4FF900539EE
:103ECF00E0C39FE5F06480F87480985003023F626E
:103EDF00AD14E5142513FFE433FEEDC39FEE6480AC
:103EEF00F87480985063ED25E0240AF582E43402DB
:103EFF00F583E0FEA3E0C39510FFEE950FFED39080
:103F0F0000A5E09F9000A4E09E503BED25E0240A21
:103F1F00F582E43402F583E0FEA3E0FF9000A2E017
:103F2F00FAA3E0FBC3EF9BEE9A401B74017E00A83F
:103F3F0005088005C333CE33CED8F9FF90053AE09C
:103F4F004EF0A3E04FF00D8089D26022C260E49062
:033F5F000539F031
:013F6200223C
:106E3B00C25330052D20162A306227C39002B4E0CE
:106E4B0094B49002B3E094005011D253900538E003
:106E5B0004F0C3940A400BD2168007C262E490057B
:046E6B0038F0A25306
:016E6F002200
:104C2800C3E5129510FFE511950FFEC3EF94B0EEA2
:104C38009404500AE5129464E51194055002D26276
:104C4800900536E024FE605514605914606A1460BB
:104C58007C24046003024CE1205F0330607B3061F8
:104C68001590053AE05455FFA3E054559002BACF89
:104C7800F0A3EFF0801390053AE054AAFFA3E054A4
:104C8800AA9002BACFF0A3EFF09002BAE0FEA3E038
:104C9800FF126C629005367402F0D25E22900536DF
:104CA8007403F022126E3B4030E4FFFE126C6290F7
:104CB80005367404F0B26122126E3B400790053647
:104CC8007405F0229005367401F0B2612290053621
:094CD8007401F0C25FC260C25E0B
:014CE10022B0
:1070C30030052220161F900537E004F0C3942D40AD
:1070D30014742DF0205E0EE4F0D25F90053A740331
:0670E300F0A374FFF0228F
:0A744000123E1F1270C3124C2822E6
:106EDA00FFD8FFE2FFECFFF60000000A00190023CA
:106EEA00002D00370041004B0055FFFBFFFCFFFD62
:106EFA00FFFEFFFFFFFF0000000100010002000388
:046F0A00000400057A
:042CD8008F828E83D6
:102CDC007E037FE8AD82AC83122833C006C007AEFA
:102CEC0083AF82C3E49FFF74109EFEAB07FAE4F936
:102CFC00F8D007D0061226379002BD1227B7E47F12
:102D0C000AFEFDFC9002BD12276AD31226FA401D62
:102D1C009002BD122751C3EF940AFFEE9400FEED12
:102D2C009400FDEC9400FC9002BD1227B79042BABF
:102D3C00E493FE740193FFE4FCFD9002BD12276A3C
:102D4C00C31226FA400D9002BB7409F0A374E3F091
:102D5C00022ECB9043AAE493FE740193FFE4FCFD96
:102D6C009002BD12276AD31226FA500D9002BB7442
:102D7C000EF0A37493F0022ECB90027CE09002BA7A
:102D8C00F025E024BAF582E43442F583E493FE7432
:102D9C000193FFE4FCFD9002BD12276AD31226FAC0
:102DAC00403D90027CE0149002BAF09002BAE0FF31
:102DBC00C39400406DEF25E024BAF582E43442F56B
:102DCC0083E493FE740193FFE4FCFD9002BD122793
:102DDC006AD31226FA404B9002BAE014F080CC90E1
:102DEC00027CE0049002BAF09002BAE0FFC394783F
:102DFC00502AEF25E024BAF582E43442F583E493BB
:102E0C00FE740193FFE4FCFD9002BD12276AD312FD
:102E1C0026FA50089002BAE004F080CC9002BAE096
:102E2C0014F09002BAE090027CF025E024BAF5820E
:102E3C00E43442F583E493FE740193FFE4FCFD90CB
:102E4C0002BD12276A12259EE47B0AFAF9F81225B4
:102E5C00ACC004C005C006C0079002BAE0FF25E074
:102E6C0024BCF582E43442F583E493FC740193FDB5
:102E7C00EF25E024BAF582E43442F583C374019360
:102E8C009DFFE4939CFEAB07FAE4F9F8D007D0065B
:102E9C00D005D004122637AB07AA0690027CE0249A
:102EAC00ECFFE434FFFE7C007D0A122514EF2BFFAF
:102EBC00EE3ACF24ABCF340A9002BBF0A3EFF090E4
:072ECC0002BBE0FEA3E0FFE2
:012ED30022DC
:10673800D2539002C3E514F0E5132514FFE433FEA9
:106748009002C3E0C39FEE6480F87480985028E0FC
:10675800FF25E02485F582E43402AB82FAEF25E0D8
:10676800240EFF7D02125B894005C253A25322907A
:0967780002C3E004F080C1A25349
:0167810022F5
:1068A600D2537A027B997D027F22125B894002C213
:1068B600537A027B9B7D027F24125B894002C2537E
:1068C6007A027B9D7D027F26125B894002C253E5D8
:1068D60013D39405400F7A027B9F7D027F28125BBB
:0768E600894002C253A253D6
:0168ED002288
:1043AC001268A64003024489900299E0FEA3E0FF44
:1043BC00122CD89000C6E02FFF9000C5E03EFEC244
:1043CC00AC900224F0A3EFF0D2AC90029DE0FEA3DF
:1043DC00E0FF7C007D11122833E47B0AFAF9F81215
:1043EC002637EF241FFFE43EFEC2AC900228F0A358
:1043FC00EFF0D2ACE513D39405402A90029FE0FE77
:10440C00A3E0FF7C007D11122833E47B0AFAF9F853
:10441C00122637EF241FFFE43EFEC2AC90022AF0B6
:10442C00A3EFF0D2AC900224E0FCA3E0FD900202DA
:10443C00ECF0A3EDF0900204ECF0A3EDF0300D3DA8
:10444C0090029BE0FEA3E0FF122CD89000C8E02F56
:10445C00FF9000C7E03EFEC2AC900226F0A3EFF046
:10446C00D2ACD3900203E09F900202E09E4006EE95
:0D447C00F0A3EFF022900204EEF0A3EFF0A9
:014489002210
:103F63009002BB1227DC000000009002BF1227DC86
:103F730000000000E4900200F0A3F09002B3741775
:103F8300F0A37470F0126738400302409A9002BAAB
:103F9300E514F0E5132514FFE433FE9002BAE0FDC7
:103FA300C39FEE6480F87480984003024071ED254E
:103FB300E02485F582E43402F583E0FEA3E0FF7C90
:103FC3000E7DD8122833C006C0079000BFE0FEA3C1
:103FD300E0FFFBAA06E4F9F8D007D00612263790D3
:103FE30002BF1227B7900200E0FEA3E0FFE4FCFD4E
:103FF3009002BF12276AD31226FA400E9002BF1214
:104003002751900200EEF0A3EFF09002B3E0FEA37D
:10401300E0FFE4FCFD9002BF12276AC31226FA50A8
:104023000E9002BF1227519002B3EEF0A3EFF020DF
:104033005E33C2AC9002BF1227519002BAE025E072
:10404300240AF582E43402F583EEF0A3EFF0D2AC58
:104053009002BB1227519002BF12276A122591903A
:1040630002BB1227B79002BAE004F0023F96205E2B
:1040730026900200E0F511A3E0F5129002B3E0F5FB
:104083000FA3E0F510C2AC9002BB12275190021EA1
:07409300EEF0A3EFF0D2AC48
:01409A002203
:104D9500E49002BFF0A3F0A3F09002C1E0FFC3943A
:104DA5000C4003024E3FEF25E024DAF582E4346E31
:104DB500F583E493FE740193FFFBAA06EA3395E0BD
:104DC500F9F89002C1E025E024DCF582E4346EF5C3
:104DD50083E493FE740193FFEE3395E0FDFC122509
:104DE50091E47B02FAF9F8126ADCE47B0AFAF9F835
:104DF5001225ACEF24ABFBEE340AFAE43DF9E43CB2
:104E0500F8900228E0FEA3E0FFE4FCFDC31226E4CF
:104E1500401F9002C1E025E024F4F582E4346EF5EC
:104E250083E493FF7401939002BFCFF0A3EFF0806A
:104E3500099002C1E004F0024D9E9002BFE0FEA37E
:024E4500E0FF8C
:014E47002248
:1035C7009002BB1227DC000000007A027BA17D027B
:1035D7007F2A125B899002A1E0FEA3E0FFEE30E4B0
:1035E7000944E09002A1F0A3EFF0124D959000C3BB
:1035F700E0FCA3E0FDC39002A2E09DFD9002A1E0E4
:103607009CCD2FFFED3EFE3395E0FDFC7B187AFC49
:1036170079FF78FF1225ACC006C0079000C1E0FE15
:10362700A3E0FFFBAA06EA3395E0F9F8D007D00636
:10363700126ADC90027D1227B790027D1227519003
:1036470002B2E025E025E0243CF582E43402F5836C
:103657001227B79002B2E004F0C394104002E4F0DE
:10366700E49002BAF09002BAE0FFC394105026A388
:1036770012276AEF25E025E0243CF582E43402F5C1
:10368700831227511225919002BB1227B79002BAD5
:10369700E004F080D0E47B10FAF9F89002BB12271F
:1036A70051126ADC9002811227B7C22BC22A9000FE
:1036B70028E0FEA3E0FFC3E49FFFE49EFE3395E00E
:1036C700FDFC90028112276AC31226E4502190055F
:1036D700F2E004F0C3940A4067740AF0D22BC2AC3C
:1036E7009002811227519002201227B7D2AC229064
:1036F7000028E0FEA3E0FFEE3395E0FDFC90028199
:1037070012276AD31226E440299005F1E004F094C9
:103717000A402D740AF0D22A7D647FA07E0F1257CB
:103727000DC2AC9002811227519002201227B7D206
:10373700AC22C2AC9002201227DC00000000D2AC01
:01374700225F
:1072DB00126CA1C25B123F631243AC305905C25909
:0472EB001235C7226F
:105AB000E49002BAF0A3F0AF14E513FDE5142DFD58
:105AC000E433FCEFC39DEC6480F8748098501DEFC4
:105AD00025E02485F582E43402F583E0FCA3E0FDB3
:105AE0009002BAEC8DF012257B0F80CD9002BAE0C7
:105AF000FEA3E0FF7C0E7DD8122833C006C00790BD
:105B000005DFE0FEA3E0FFFBAA06E4F9F8D007D02A
:0C5B1000061226379000BFEEF0A3EFF065
:015B1C002266
:106D55009000C3E0FEA3E0FFC39002A2E09FFF9076
:106D650002A1E09EFE3395E0FDFC7B187AFC79FFDD
:106D750078FF1225AC9005D612276A126ADCEF4E11
:0A6D850060089000C1EEF0A3EFF0EB
:016D8F0022E1
:10740A009002A1E0FFA3E09000C3CFF0A3EFF02227
:106A0E00900299E0FEA3E0FF122CD8C39005DCE0C3
:106A1E009FFF9005DBE09EFE9000C5E0FCA3E0FD2D
:106A2E00C3EF9DFDEE9CFCC3ED9496EC64809480C8
:106A3E005012ED946AEC6480947F40089000C5EE8D
:046A4E00F0A3EFF0D2
:016A52002221
:106A530090029BE0FEA3E0FF122CD8C39005DEE07A
:106A63009FFF9005DDE09EFE9000C7E0FCA3E0FDE4
:106A7300C3EF9DFDEE9CFCC3ED9496EC6480948083
:106A83005012ED946AEC6480947F40089000C7EE46
:046A9300F0A3EFF08D
:016A970022DC
:106A98009005E1E0900497F09005E2E0900498F00A
:106AA8009005E3E0900499F09005E4E090049AF0F2
:106AB8009005E5E090049BF09005E6E090049CF0DA
:106AC8009005E7E090049DF07E047F9712518DD2E7
:046AD8003AD23D224F
:1063950030794BC2799005DAE030E003125AB090BB
:1063A50005DAE030E403126D559005DAE030E503D7
:1063B50012740A9005DAE030E203126A0E9005DAEB
:1063C500E030E303126A539005DAE030E703126A1E
:0F63D50098E49005DAF0D2709005F57402F0228A
:10652000306A0DC26AD268E49005F4F01273282232
:1065300030683A12723F203134900087E075F002E3
:10654000A4FFAEF09005F4E004F0C39FEE6480F881
:106550007480984018C268E4F012733B307602C22F
:0E65600019C21BC21C301505C215126CDE22BA
:1068150030690DC269D267E49005F3F01273022264
:1068250030673512723F20302F900087E075F002F7
:10683500A4FFAEF09005F3E004F0C39FEE6480F88A
:106845007480984013C267E4F0127315307507C25F
:0968550018C214126CDEC21A22F2
:1071B200300719303B119003E7E004F0C394054017
:0D71C2000BD2397405F022E49003E7F022AF
:105E52009002E4EEF0A3EFF0A3EDF0A3EAF0A3EBDF
:015E6200F04F
:105E6300C253203941E4A3F09002E4E0FCA3E0FD37
:105E7300A3E09002FAF0E4A3F09002E7E0FFA3E0CE
:105E83009002FCCFF0A3EFF07B017FA0123CD8502F
:105E930004D25380117F011269369002E9E004F0C5
:0D5EA300E0C3940540C2A253B3923BA2534A
:015EB00022CF
:105EB1009002C6EEF0A3EFF0A3EDF0A3EAF0A3EB9E
:015EC100F0F0
:105EC200C254203941E4A3F09002C6E0FCA3E0FDF5
:105ED200A3E09002F0F0E4A3F09002C9E0FFA3E097
:105EE2009002F2CFF0A3EFF07B017FA012325B5061
:105EF20004D25480117F011269369002CBE004F083
:0D5F0200E0C3940540C2A254B3923BA254E8
:015F0F00226F
:105B1D007E027FBD7B08E4FD127025E49002BBF090
:105B2D00A3F09002BBE0FEA3E0FFE4FCFD7BFF7A57
:105B3D0007F9F8D31226E4402E53B1F89002BBE0DA
:105B4D00FEA3E07805C333CE33CED8F9241FFFE48E
:105B5D003EFE7A027BBD7D01125E529002BBE47562
:105B6D00F00112257B80BB7A027BBD7D087FE07E34
:0B5B7D00FF125E52E49003E0F0A3F082
:015B880022FA
:10578E00C2537A027BBA7D087FE07EFF125EB19231
:10579E00539002BBE0FF9002BAE02F9002BCF09053
:1057AE0002BFE0FF9002BEE02F9002C0F09002BD5B
:1057BE00E0FF9002BCE0B507179002BAE0FEA3E04E
:1057CE007C002400FFEC3E9003E0F0A3EFF0802A73
:1057DE009002C1E0FF9002C0E0B507179002BEE054
:1057EE00FEA3E07C002400FFEC3E9003E0F0A3EF6C
:0C57FE00F08007E49003E0F0A3F0A25359
:01580A00227B
:10665400E49002C4F07E047F971230997E047F9701
:106664007C027DBB7B07126F0EE4FF74BB2FF582A7
:10667400E43402F583E0FE9002C4E02EF00FEFB4A0
:1066840007E99002C4E09002C2F0A3745AF07A02BF
:0B6694007BBB7D097FF07EFF125E5291
:01669F0022D8
:106B62009003E0E0FCA3E0FDEC9002DCF0AF05A3B3
:106B7200EFF09002DCE02F9002DFF09002DCE09078
:106B820002E0F09002DDE09002E1F09002DFE0909E
:106B920002E3F07A027BDC7D087FE07EFF125E5228
:016BA20022D0
:053414009002BBEFF087
:103419006410701A7E037FE87C027DBC7B03126F07
:103429000E7E037FEC7C027DBF126F0E801F7E042F
:103439007F971230997E047F977C027DBC7B0312B3
:103449006F0E7E047F9A7C027DBF126F0E9002067A
:10345900E0FCA3E0FDEC9002C2F0A3EDF0900208BD
:10346900E0FCA3E0FDEC9002C4F0A3EDF090022C87
:10347900122751781812270B9002C6EFF090022CF0
:10348900122751781012270B9002C7EFF090022CE7
:10349900122751780812270B9002C8EFF090022CDE
:1034A9001227519002C9EFF0900230122751781873
:1034B90012270B9002CAEFF09002301227517810B0
:1034C90012270B9002CBEFF09002301227517808A7
:1034D90012270B9002CCEFF0900230122751900284
:1034E900CDEFF090021EE0FCA3E0FDAE047818CE0B
:1034F900C313CE13D8F99002CEF0EDAE047810CEF6
:10350900C313CE13D8F99002CFF090021EE0FCA3AA
:10351900E0FDEC9002D0F0A3EDF0900220122751CB
:10352900781812271E9002D2EFF09002201227512C
:10353900781012271E9002D3EFF090022012275123
:10354900780812271E9002D4EFF09002201227511A
:103559009002D5EFF0900224E0FCA3E0FDEC90028C
:10356900D6F0A3EDF0900236E0FCA3E0FDEC90026A
:10357900D8F0A3EDF09002BBE09002DAF0A3745A00
:10358900F09003E0E0FEA3E0FF7A027BBC7D20120D
:103599005E529003E0E475F02012257B9003E0E091
:1035A900FEA3E0FFE4FCFD7BE07AFFF9F8D31226E5
:0D35B900E45007E49003E0F0A3F0126B6211
:0135C60022E2
:105BF4009003F2E02480FFE434FFEF7D00C454F00E
:105C0400FC900401E02488FFE434FFFEEF7807C32E
:105C140033CE33CED8F92DFFEE3CFE900402E0FDE6
:105C24007A047B03125EB17B017A0479009004024A
:105C3400E02403FD127209900402E02403F582E4D7
:105C44003404F583EFF0C29C9003FAE02400F5825B
:0A5C5400E43404F583E0F599D2A0D2
:015C5E002223
:1058F5009003F2E02480FFE434FFEF7D00C454F010
:10590500FC9004A1E02488FFE434FFFEEF7807C390
:1059150033CE33CED8F92DFFEE3CFE9004A2E0FD48
:105925007A047BA3125EB17B017A0479A09004A26C
:10593500E02403FD1272099004A2E024A3F582E499
:105945003404F583EFF0758640C2A49003FBE02490
:0E595500A0F582E43404F583E0F5A1E4F586C4
:015963002221
:105964009003F2E02480FFE434FFEF7D00C454F0A0
:10597400FC900541E02488FFE434FFFEEF7807C380
:1059840033CE33CED8F92DFFEE3CFE900542E0FD38
:105994007A057B43125EB17B017A0579409005421A
:1059A400E02403FD127209900542E02443F582E4E9
:1059B4003405F583EFF0758640C2949003FCE0242F
:0E59C40040F582E43405F583E0F591E4F586C4
:0159D20022B2
:1068EE007E047F971230997E047F977C047D037B14
:1068FE0007126F0E7B017A047900900402E02403E4
:10690E00FD127209900402E02403F582E43404F5CA
:10691E0083EFF0C29C9003FAE02400F582E4340485
:08692E00F583E0F599D2A022E7
:1066A0007E047F971230997E047F977C047DA37BC4
:1066B00007126F0E7B017A0479A09004A2E02403F4
:1066C000FD1272099004A2E024A3F582E43404F5DB
:1066D00083EFF0758640C2A49003FBE024A0F5820E
:0C66E000E43404F583E0F5A1E4F5862223
:1066EC007E047F971230997E047F977C057D437BD7
:1066FC0007126F0E7B017A057940900542E0240366
:10670C00FD127209900542E02443F582E43405F54C
:10671C0083EFF0758640C2949003FCE02440F58230
:0C672C00E43405F583E0F591E4F58622E5
:104E4800200703024EF3203A03024EF3C23A3038E9
:104E580005C238125B1D9003E2E0FF7008A3E07002
:104E680004A3E06021EF6008E49003E2F0125BF431
:104E78009003E3E06005E4F01259649003E4E06015
:104E880005E4F01259649003EFE0FF7008A3E070A6
:104E980004A3E06021EF6008E49003EFF01268EEED
:104EA8009003F0E06005E4F01266A09003F1E06082
:104EB80005E4F01266EC303D05C23D126654303C04
:104EC8000CC23C9002BA7410F0FF12341430420C39
:104ED800C2429002BA7401F0FF123414303F0CC27F
:0B4EE8003F9002BA7402F0FF12341475
:014EF300229C
:1045610020070302463390002EE0FF9003DDE004B4
:10457100F0C39F4009E4F07E047F971230999003C5
:10458100DEE475F00112257BFEC3E5F09410EE9494
:104591000E400BE49003DEF0A3F0D23AD23D202A84
:1045A1001ED241304006C240D23AD24230190B30BD
:1045B1003E08C23ED23AD23F8005201902D23E3097
:1045C100416990002CE0FEA3E0FFEE3395E0FDFC95
:1045D10090022012276AC31226E4404F9003E5E0BF
:1045E1007002A3E070147E047F971230997E047FDD
:1045F100977C037DE87B07126F0E90002BE0FF7E16
:10460100007C007D3C1225149003E5E475F0011255
:10461100257BFCD3E5F09FEC9E4017E49003E5F089
:10462100A3F0D240C241D23AD23C22E49003E5F059
:03463100A3F022D1
:031053000259D36C
:1059D300C0E0C083C082C0D075D000C007C0867548
:1059E300860030D807C2D87F0112102E30D907C2E3
:1059F300D97F0212102E30DA07C2DA7F0412102E7A
:105A030030DB07C2DB7F0812102E30DC07C2DC7FDD
:105A13001012102E30DD07C2DD7F2012102E30DE73
:105A230007C2DE7F4012102E30DF07C2DF7F8012F5
:0F5A3300102ED086D007D0D0D082D083D0E032D2
:03102B00021003AD
:10100300C0E0C083C082C0D0C086758640C28F75E1
:10101300860012710FD086D0D0D082D083D0E03238
:10504A00307A030250EB75090F20A7057509018014
:10505A000620B003750902E509650C6038050EE5FE
:10506A000E7002050DC3E50B940AE50A940040652B
:10507A00E50E940AE50D94004067E50B9490E50A65
:10508A0094014008E50C4440F5088003850C08D2D9
:10509A007A80428040E509640F6037E4F50DF50E29
:1050AA00050BE50B7002050AB4900EE50AB4010976
:1050BA00E50C4410F508D27A22E50BB4B023E50AD0
:1050CA00B4041E750A01750B90E50C4420F508D24C
:1050DA007A2275080FE4F50AF50BF50DF50E850928
:0150EA000CB9
:0150EB0022A2
:106E7000AB07AA06C2AF43A701EAF5F7AF038FFB42
:106E8000AF058FFC75F26E75F30575F40A75F5099B
:106E9000EAADF7B50509E475F606000000000053F9
:056EA000A7FED2AF22A5
:1070E900D256E4FDFCEF2DFBEE3C8B82F583E49355
:1070F9006004C256800D0DBD00010CE4B505E6EC37
:05710900B402E2A256F1
:01710E00225E
:0860DE009002C0EEF0A3EFF008
:1060E600D256AE04AF05E4A3F0A3F09002C2E0FCE2
:1060F600A3E0FDC3EC940250369002C1E02DFD9062
:1061060002C0E03C8D82F583E493FD9002C2E0FA82
:10611600A3E02FF582EE3AF583E0FCED6C6004C255
:1061260056800C9002C2E475F00112257B80BCA259
:016136005612
:016137002245
:085472009002C0EEF0A3EFF080
:10547A00C256AF05A3ECF0A3EFF0E4FDFC9002C026
:10548A00E0FAA3E0FB2DF5FBEB2DEA3CF5F7A3E0F0
:10549A00FEA3E02DF582EE3CF583E0F5FC75F26E95
:1054AA0020AF3D75F305E5A7603275F40A9005F65D
:1054BA00E06455702375F5099002C1E02D9002C091
:1054CA00E03CABF7B5030DE475F6060000000000FA
:1054DA00D2568010C2568019C2568015C256801103
:1054EA00C256800D0DBD00010CED7003EC64027014
:0354FA008CA2562B
:0154FD00228C
:0E52C0009002BCEEF0A3EFF0A3ECF0A3EDF033
:1052CE00C25553B1F8C2AF43A7019002BCE0FF7EB6
:1052DE0000F5F775F2E620AF5B75F305E5A76054B0
:1052EE0075F40A9005F6E06455704975F509ADF749
:1052FE00EF6D7001EE703D75F60600000000009037
:10530E0002BCE0FEA3E0FF1270E950289002BCE060
:10531E00FEA3E0FFA3E0FCA3E0FD12547250159033
:10532E0002BCE0FEA3E0FFA3E0FCA3E0FD1260DE02
:10533E005002D255E4F5F2F5F3F5F4F5F5F5F65322
:08534E00A7FEF5F7D2AFA2554E
:015356002234
:1047BB00C253C254206F0302487BC26F9005F6743C
:1047CB0055F0E513D39405400C9002BA7427F0A36F
:1047DB007410F0800A9002BA7413F0A37488F090EE
:1047EB0002BAE0FEA3E0FFC390021FE09F90021EFF
:1047FB00E09E406B9001FEE0645A7004A3E064A558
:10480B00705DFDFCFFFE1252C04023E4FDFCFFFE79
:10481B001252C04019D25374FF9001FEF0A3F0FD69
:10482B007FFE7E01126E707DFF7FFF126E70E4FDC6
:10483B00FCFF7E021252C0402AE4FDFCFF7E0212F6
:10484B0052C0401FD25474FF9001FEF0A3F0FD7FC5
:10485B00FE7E03126E707DFF7FFF126E708004D29E
:10486B0053D254E49005F6F0305305305402D26E17
:01487B00221A
:0E5F10009002BAEEF0A3EFF0A3EAF0A3EBF0DC
:105F1E00D253AE04AF058E198F1AC2AF43A70153E9
:105F2E00B1F8E4FFFED39002BDE09F9002BCE09E6C
:105F3E0040279002BBE02FFD9002BAE03E8D82F525
:105F4E0083E493851A82851983F0051AE51A700287
:105F5E0005190FBF00010E80CC53A7FED2AFA2537E
:015F6E002210
:1072C6003070119005F5E004F0C394024006C270D8
:0572D600E4F0D26F227C
:10704F00C25343A701EEC313FEEF1325E0FFEE3348
:10705F008F82F583740193B4A507E493B45A02D2D7
:06706F005353A7FEA253DB
:0170750022F8
:056F71009002BAEFF0F0
:106F7600758640758830AE04AF057C1F7D401228AB
:106F860033E4FB7A01F9F8122637C3E49FFFE49E47
:0A6F9600FE8F8CF58DD28AE4F5869B
:016FA00022CE
:057133009002BAEFF02C
:10713800A2AFE433FFC2AF43B20800000000000072
:0C714800000053B26043B20424FF92AF79
:017154002218
:10560B009005EBEEF0A3EFF0A3EDF075C7B09005AE
:10561B00EBE0FEA3E0FFFBAA06E4F9F87FD87EB827
:10562B007D05FC126ADC8FCC9005EBE0FEA3E0FF5E
:10563B00FBAA06E4F9F87FD87EB87D05FC126ADC7C
:10564B00780812271E8FCDAFCDEFFEADCC7C00E4DA
:10565B002DFFEC3EFE9005EDE0FBFD1225147D6465
:10566B001225268FCEAFCDEFFEADCC7C00E42DFF07
:10567B00EC3EFEAD031225147D64122526EEF5CF0C
:01568B0022FC
:10568C009005EEEEF0A3EFF0A3EDF075B6B090053B
:10569C00EEE0FEA3E0FFFBAA06E4F9F87FD87EB8A3
:1056AC007D05FC126ADC8FAE9005EEE0FEA3E0FFF8
:1056BC00FBAA06E4F9F87FD87EB87D05FC126ADCFB
:1056CC00780812271E8FAFAFAFEFFEADAE7C00E4B3
:1056DC002DFFEC3EFE9005F0E0FBFD1225147D64E1
:1056EC001225268FA4AFAFEFFEADAE7C00E42DFFEC
:1056FC00EC3EFEAD031225147D64122526EEF5A5B5
:01570C00227A
:10570D009002BFEEF0A3EFF0A3EDF075B7B09002ED
:10571D00BFE0FEA3E0FFFBAA06E4F9F87FD87EB850
:10572D007D05FC126ADC8FBC9002BFE0FEA3E0FF9A
:10573D00FBAA06E4F9F87FD87EB87D05FC126ADC79
:10574D00780812271E8FBDAFBDEFFEADBC7C00E407
:10575D002DFFEC3EFE9002C1E0FBFD1225147D6491
:10576D001225268FBEAFBDEFFEADBC7C00E42DFF34
:10577D00EC3EFEAD031225147D64122526EEF5BF19
:01578D0022F9
:10693600E5B2547070067C067D868020E5B2547000
:10694600FEBE20067C037D438012E5B25470FEBE77
:1069560040067C017DA180047C007D8BE4FEEEC3B5
:106966009F5014E4FBFAC3EB9DEA9C50070BBB0057
:07697600010A80F20E80E728
:01697D0022F7
:105CC50090002FE0645A705A900061E0645A705257
:105CD500900073E0645A704A900088E0645A7042FC
:105CE50090008DE0645A703A900098E0645A7032E2
:105CF5009000A1E0645A702A9000A9E0B45A23905C
:105D050000BAE0B45A1C9000BEE0B45A159000CA1F
:105D1500E0B45A0E9001FEE0645A7004A3E064A555
:065D25006002C322D3223C
:087025009002C6EEF0A3EFF0AB
:10702D00E4FFEFC39B501A9002C6E0F8A3E0F5828F
:10703D008883EDF09002C6E475F00112257B0F8078
:01704D00E161
:01704E00221F
:086F0E009002DCEEF0A3EFF0AD
:106F1600E4FFEFC39B50239002DCE0F8A3E0F58288
:106F26008883E08D828C83F00DBD00010C9002DC1D
:0A6F3600E475F00112257B0F80D8EE
:016F4000222E
:0C742800758E5543870100000000002213
:0C743400758E5543870200000000002206
:106FCE009005EAE064127023204306204403304506
:106FDE001A207017206F14C2AFE4F5A8F5A9F58832
:0C6FEE00F5E8F59DF59CF59812000022D6
:10678200D228D229201403301602C22820110F2049
:10679200130C201B09201C06201503301602C229E7
:1067A200202B0E201009201206201803301A02C2D4
:1067B20028202A05301902C229201B06201C03307A
:0A67C2001502C228301A02C2292273
:106FA100126782A273302801B34008A2743029010C
:106FB100B35019A2289273A2299274A229E433FF33
:0D6FC10025E0FFA228E4334FFF1272B12239
:10697E00201844C3900063E09512900062E09511D8
:10698E00501F9003BFE475F00112257BFEC3E5F0A6
:10699E009401EE94004020D218E49003BFF0A3F0CF
:1069AE0022D3900065E09512900064E095114007A7
:0869BE00E49003BFF0A3F022F6
:1069C600201944D3900075E09510900074E0950F5F
:1069D600401F9003C1E475F00112257BFEC3E5F06C
:1069E6009401EE94004020D219E49003C1F0A3F084
:1069F60022C3900077E09510900076E0950F50073F
:086A0600E49003C1F0A3F022AB
:1063E40020104B90008EE0FEA3E0FF900204E0FC3E
:1063F400A3E0FDD39FEC9E401F9003D1E475F00110
:1064040012257BFEC3E5F09401EE94004020D210E7
:10641400E49003D1F0A3F022900090E0FEA3E0FF0B
:0F642400C3ED9FEC9E5007E49003D1F0A3F0224C
:1064330020124B900092E0FEA3E0FF900202E0FCEA
:10644300A3E0FDC39FEC9E501F9003D5E475F001BC
:1064530012257BFEC3E5F09401EE94004020D21296
:10646300E49003D5F0A3F022900094E0FEA3E0FFB4
:0F647300D3ED9FEC9E4007E49003D5F0A3F022F9
:1064820020114B900099E0FEA3E0FF900204E0FC93
:10649200A3E0FDD39FEC9E401F9003D3E475F0016F
:1064A20012257BFEC3E5F09401EE94004020D21148
:1064B200E49003D3F0A3F02290009BE0FEA3E0FF60
:0F64C200C3ED9FEC9E5007E49003D3F0A3F022AC
:1064D10020134B90009DE0FEA3E0FF900202E0FC40
:1064E100A3E0FDC39FEC9E501F9003D7E475F0011C
:1064F10012257BFEC3E5F09401EE94004020D213F7
:10650100E49003D7F0A3F02290009FE0FEA3E0FF08
:0F651100D3ED9FEC9E4007E49003D7F0A3F02258
:106D9000307B37123F631243AC12697E1269C61210
:106DA00063E41264331264821264D190053FE004FC
:106DB000F0C394024014C27B205A0920390620787F
:0B6DC00003306E03D26322123A20223F
:1046340020185C201459C3900063E0951290006226
:10464400E095115033900066E075F00AA4FFAEF0D7
:104654009003BFE475F00112257BFCC3E5F09FECE9
:104664009E50030246F7D218C275E49003BFF0A32C
:10467400F09003D9F0A3F022D3900065E095129056
:104684000064E09511406CE49003BFF0A3F0222095
:104694007561D3900065E09512900064E095114037
:1046A4003C900067E075F00AA4FFAEF09003D9E4F3
:1046B40075F00112257BFCC3E5F09FEC9E4034307D
:1046C4000E06D275D2698007C218C214126CDEE4D9
:1046D4009003BFF0A3F09003D9F0A3F022C390009D
:1046E40063E09512900062E095115007E49003D9BD
:0446F400F0A3F0221D
:10487C00201959D3900075E09510900074E0950FB5
:10488C004033900078E075F00AA4FFAEF09003C1BD
:10489C00E475F00112257BFCC3E5F09FEC9E500300
:1048AC00024937D219C276E49003C1F0A3F0900309
:1048BC00DBF0A3F022C3900077E09510900076E037
:1048CC00950F5067E49003C1F0A3F02220765CC3EF
:1048DC00900077E09510900076E0950F503790009F
:1048EC0079E075F00AA4FFAEF09003DBE475F001FB
:1048FC0012257BFCC3E5F09FEC9E402F300F06D2B7
:10490C0076D26A8002C219E49003C1F0A3F090033E
:10491C00DBF0A3F022D3900075E09510900074E0CA
:0C492C00950F4007E49003DBF0A3F0229D
:1049380020105E90008EE0FEA3E0FF900204E0FCF1
:10494800A3E0FDD39FEC9E4031900096E075F014F3
:10495800A4FFAEF09003D1E475F00112257BFAC3F1
:10496800E5F09FEA9E50030249F3D210E49003D188
:10497800F0A3F09003C3F0A3F022900090E0FEA310
:10498800E0FFC3ED9FEC9E5062E49003D1F0A3F0EA
:1049980022900090E0FEA3E0FF900204E0FCA3E078
:1049A800FDC39FEC9E502E900096E075F014A4FF76
:1049B800AEF09003C3E475F00112257BFAC3E5F06D
:1049C8009FEA9E4026C210E49003D1F0A3F0900322
:1049D800C3F0A3F02290008EE0FEA3E0FFD3ED9F8A
:0C49E800EC9E4007E49003C3F0A3F02213
:1049F40020125E900092E0FEA3E0FF900202E0FC31
:104A0400A3E0FDC39FEC9E5031900096E075F01436
:104A1400A4FFAEF09003D5E475F00112257BFAC330
:104A2400E5F09FEA9E5003024AAFD212E49003D508
:104A3400F0A3F09003C7F0A3F022900094E0FEA34B
:104A4400E0FFD3ED9FEC9E4062E49003D5F0A3F029
:104A540022900094E0FEA3E0FF900202E0FCA3E0B9
:104A6400FDD39FEC9E402E900096E075F014A4FFB9
:104A7400AEF09003C7E475F00112257BFAC3E5F0AC
:104A84009FEA9E4026C212E49003D5F0A3F090035F
:104A9400C7F0A3F022900092E0FEA3E0FFC3ED9FD5
:0C4AA400EC9E5007E49003C7F0A3F02242
:104AB00020115E900099E0FEA3E0FF900204E0FC6C
:104AC000A3E0FDD39FEC9E4031900096E075F0147A
:104AD000A4FFAEF09003D3E475F00112257BFAC376
:104AE000E5F09FEA9E5003024B6BD211E49003D392
:104AF000F0A3F09003C5F0A3F02290009BE0FEA38A
:104B0000E0FFC3ED9FEC9E5062E49003D3F0A3F06E
:104B10002290009BE0FEA3E0FF900204E0FCA3E0F3
:104B2000FDC39FEC9E502E900096E075F014A4FFFC
:104B3000AEF09003C5E475F00112257BFAC3E5F0F1
:104B40009FEA9E4026C211E49003D3F0A3F09003A5
:104B5000C5F0A3F022900099E0FEA3E0FFD3ED9F03
:0C4B6000EC9E4007E49003C5F0A3F02297
:104B6C0020135E90009DE0FEA3E0FF900202E0FCAB
:104B7C00A3E0FDC39FEC9E5031900096E075F014BD
:104B8C00A4FFAEF09003D7E475F00112257BFAC3B5
:104B9C00E5F09FEA9E5003024C27D213E49003D712
:104BAC00F0A3F09003C9F0A3F02290009FE0FEA3C5
:104BBC00E0FFD3ED9FEC9E4062E49003D7F0A3F0AE
:104BCC002290009FE0FEA3E0FF900202E0FCA3E035
:104BDC00FDD39FEC9E402E900096E075F014A4FF40
:104BEC00AEF09003C9E475F00112257BFAC3E5F031
:104BFC009FEA9E4026C213E49003D7F0A3F09003E3
:104C0C00C9F0A3F02290009DE0FEA3E0FFC3ED9F4E
:0C4C1C00EC9E5007E49003C9F0A3F022C6
:10613800201A5590006D12275190027D12276AD3BC
:106148001226E4402A900071E075F00AA4FFAEF030
:106158009003CDE475F00112257BFCC3E5F09FECBC
:106168009E4025D21AD269E49003CDF0A3F02220F4
:106178006716D39003CEE094009003CDE0940040DE
:096188000774FFF5F012257B22DB
:10619100201B5590007D12275190027D12276AC362
:1061A1001226E4502A900081E075F00AA4FFAEF0B7
:1061B1009003BBE475F00112257BFCC3E5F09FEC75
:1061C1009E4025E49003BBF0A3F0D21BD26A2220AB
:1061D1006816D39003BCE094009003BBE0940040A8
:0961E1000774FFF5F012257B2282
:1061EA00201C5590008212275190027D12276AC303
:1061FA001226E4502A900086E075F002A4FFAEF061
:10620A009003BDE475F00112257BFCD3E5F09FEC09
:10621A009E4025E49003BDF0A3F0D21CD26A22204E
:10622A006816D39003BEE094009003BDE09400404A
:09623A000774FFF5F012257B2228
:10717500207B1B12463412487C1249381249F412FE
:0F7185004AB0124B6C1261381261911261EA220A
:10580B00300272201B06201C03301539900072E009
:10581B0075F014A4FFAEF09003CFE475F0011225E0
:10582B007BFCC3E5F09FEC9E401BE49005F4F090ED
:10583B0003CFF0A3F0C21BC21CC26AC268301505AD
:10584B00C215126CDE301A2D900072E075F014A4A4
:10585B00FFAEF09003CBE475F00112257BFCD3E592
:10586B00F09FEC9E400FE49003CBF0A3F0C21A9094
:06587B0005F3F0C26722F4
:1071CF00300719307711900496E004F0C39405400E
:0D71DF000BD2787405F022E4900496F022A3
:0E6028009002F1EFF0A3EDF0A3EAF0A3EBF08D
:10603600C256207840E4A3F09002F1E0FD7C00A374
:10604600E09002FAF0E4A3F09002F3E0FFA3E09000
:1060560002FCCFF0A3EFF0E4FB7FDE123CD8500445
:10606600D25680117F011269369002F5E004F0E005
:0C607600C3940540C3A256B39277A25613
:0160820022FB
:0E6083009002E7EFF0A3EDF0A3EAF0A3EBF03C
:10609100C255207840E4A3F09002E7E0FD7C00A324
:1060A100E09002F0F0E4A3F09002E9E0FFA3E090B9
:1060B10002F2CFF0A3EFF0E4FB7FDE12325B50047B
:1060C100D25580117F011269369002EBE004F0E0B5
:0C60D100C3940540C3A255B39277A255BA
:0160DD0022A0
:083099009002DCEEF0A3EFF061
:1030A100C2547A027BDE7D09E4FF12608340030291
:1030B10032589002E5E030E00302324B9002E0E04A
:1030C10020E70302316A9002DEE0FF547094504021
:1030D1000302316AEF540F9409400302316AE0544C
:1030E1007F9459400302316AA3E0FF547094505019
:1030F10078EF540F94095071E0547F9459506AA3AA
:10310100E0FF543094205061EF540F9409505AE07D
:10311100542F94245053A3E0FF54309430504AEF7D
:10312100540F94095043E0543FFF9431503BEF60FA
:1031310038A3E0FF54109410502FEF540F9409500E
:1031410028E0541FFF94125020EF601DA3E0FF54AC
:10315100F094905014EF540F9409500DE09499504D
:1031610008A3E05407940640779002DCE0FEA3E058
:10317100FFF5828E83E09002DEF08F828E83A3E0E2
:103181009002DFF09002DCE0A3E0F5828E83A3A33E
:10319100E09002E0F08F828E83A3A3A3E09002E18E
:1031A100F09002DCE0A3E02404F582E43EF583E044
:1031B1009002E2F0EF2405F582E43EF583E090020F
:1031C100E3F09002DCE0A3E02406F582E43EF5831F
:1031D100E09002E4F07E027FDE12518D92548077FE
:1031E1009002DEE0FF9002DCE0FCA3E0FDF5828CC2
:1031F10083EFF09002DFE08D828C83A3F09002E0F8
:10320100E0541F8D828C83A3A3F09002E1E08D82B4
:103211008C83A3A3A3F09002E2E0FFED2404F582E6
:10322100E43CF583EFF09002E3E0FFED2405F58245
:10323100E43CF583EFF09002E4E0FFED2406F58233
:10324100E43CF583EFF0D254800D9002DCE0FEA364
:09325100E0FF12518D9254A254C9
:01325A002251
:08518D009002E7EEF0A3EFF041
:10519500C255A37490F07A027BE97D017F07126006
:1051A5002892559002E7E0FEA3E0FFF5828E83E0AA
:1051B5009002EAF08F828E83A3E09002EBF09002DA
:1051C500E7E0FCA3E0FDF5828C83A3A3E044809097
:1051D50002ECF08D828C83A3A3A3E09002EDF09006
:1051E50002E7E0A3E0FF2404F582E43EF583E090C6
:1051F50002EEF0EF2405F582E43EF583E09002EF40
:10520500F09002E7E0A3E02406F582E43EF583E0B2
:105215009002F0F07A027BEA7D07E4FF12602892A3
:0352250055A2553A
:015228002263
:0853E5009002BAEEF0A3EFF014
:1053ED00C253E49002C5F07E027FBC7B09FD1270B2
:1053FD00257A027BBC7D097FF07EFF125EB1E4FF52
:10540D0074BC2FF582E43402F583E0FE9002C5E012
:10541D002EF00FEFB407E99002C5E0FF9002C3E054
:10542D00B50706A3E0645A601BE49002BCF0A3F03C
:10543D00A37412F0A37401F0A37405F0A37420F00B
:10544D00A37405F07E027FBC9002BAE0FCA3E0FDE0
:10545D007B07126F0E9002BAE0FEA3E0FF123099A7
:04546D009253A25361
:015471002218
:1041BA0000070E091C1B1215383F363124232A2DFD
:1041CA0070777E796C6B6265484F464154535A5DED
:1041DA00E0E7EEE9FCFBF2F5D8DFD6D1C4C3CACDDD
:1041EA0090979E998C8B8285A8AFA6A1B4B3BABDCD
:1041FA00C7C0C9CEDBDCD5D2FFF8F1F6E3E4EDEABD
:10420A00B7B0B9BEABACA5A28F88818693949D9AAC
:10421A002720292E3B3C35321F18111603040D0A9C
:10422A005750595E4B4C45426F68616673747D7A8C
:10423A00898E878095929B9CB1B6BFB8ADAAA3A47C
:10424A00F9FEF7F0E5E2EBECC1C6CFC8DDDAD3D46C
:10425A00696E676075727B7C51565F584D4A43445C
:10426A00191E171005020B0C21262F283D3A33344C
:10427A004E49404752555C5B7671787F6A6D64633C
:10428A003E39303722252C2B0601080F1A1D14132C
:10429A00AEA9A0A7B2B5BCBB9691989F8A8D84831C
:1042AA00DED9D0D7C2C5CCCBE6E1E8EFFAFDF4F30C
:10720900E4FFEDD3940040131224FB6F9041BA932D
:0B721900FF740129F9E43AFA1D80E738
:017224002247
:10707600D2587D807CBBE5C820E31053B1F8ED4CB7
:107086006009ED1D70011C80ED80EBE5D154F86FB1
:067096006002C258A2587E
:01709C0022D1
:103CD8009002F9EBF09002F6EFF0A3ECF0A3EDF010
:103CE800D25790030274BBF0A37480F09002FEEFE9
:103CF800F0A3EDF09002FCE0FEA3E0F5828E83E0F5
:103D0800900300F07B017A0279FE7D03127209901C
:103D18000301EFF09002FAE0D394005003023E1C36
:103D280043E6C043D10143C80175C8607F081270DB
:103D380076400C7F101270764005C257023DF9900C
:103D480002F6E0F58D75C8407F181270764005C2FE
:103D580057023DF99002F9E0B401159002F7E0F539
:103D68008D75C8407F281270764005C257023DF90C
:103D78009002F7E0A3E0F58D75C8407F28127076B1
:103D88004004C257806B9002FBE06401702EA3E0F0
:103D9800FEA3E0F5828E83E0F58D75C8407F28127A
:103DA80070764004C2578049900301E0F58D75C8CC
:103DB800407F281270764039C2578035E4FE900261
:103DC800FAE0FFEEC39F50299002FCE0FCA3E0F567
:103DD800828C83E0F58D75C8407F28127076400488
:103DE800C257800D9002FCE475F00112257B0E800D
:103DF800CD75C850E5C830E41B53B1F8900302E014
:103E08007002A3E0600E90030274FFF5F012257BA8
:063E180080E280E0A257E9
:013E1E002281
:0A325B00AA079002EDECF0A3EDF0DD
:10326500D256E4900323F0A374BBF0A37480F090CE
:1032750002F5EAF0A3EDF0EA4401A3F09002F0E0D4
:10328500D39400500302341143E6C043D10143C82F
:103295000175C8607F08127076400C7F1012707639
:1032A5004005C2560233EE8A8D75C8407F181270EC
:1032B500764005C2560233EEEBB401159002EDE0FF
:1032C500F58D75C8407F281270764005C2560233C9
:1032D500EE9002EDE0A3E0F58D75C8407F281270F1
:1032E500764005C2560233EE75C8607F08127076C7
:1032F500400C7F101270764005C2560233EEEA4448
:1033050001F58D75C8407F401270764005C25602A2
:1033150033EEE49002F4F09002F0E0FF9002F4E066
:10332500FEC39F50579002F1E07031EF14B5060AC5
:1033350075C8407F58127076800875C8447F501252
:1033450070769002F2E0FEA3E0F5828E83E58DF0C3
:103355009002F2E475F00112257B801875C8447F50
:10336500501270769002F4E024F8F582E43402F508
:1033750083E58DF09002F4E004F0809B9002F1E08B
:103385006401706575C8407F58127076900323E517
:103395008DF07B017A0279F59002F0E02403FD12AD
:1033A5007209900323E0B5073EE49002F4F0900221
:1033B500F0E0FF9002F4E0FEC39F502D74F82EF567
:1033C50082E43402F583E0FF9002F2E0FCA3E0F52D
:1033D500828C83EFF09002F2E475F00112257B9068
:1033E50002F4E004F080C7C25675C850E5C830E461
:1033F5001B53B1F8900324E07002A3E0600E900324
:0E3405002474FFF5F012257B80E280E0A256D1
:013413002296
:10726E0075C632E4F5E6F5D1758A2075D10275C87A
:07727E00407589FFF58D2228
:035DF10075C43244
:105DF400E4F5877598509002BA747FF0A374CCF0E0
:105E04009002BAE0F59D759CCCE0FEA3E0FFFBE4B4
:105E1400C39BFF74809EFEE49400FDE49400FCE4C4
:105E24007B10FAF9F81225ACEC12243CA804A9055D
:105E3400AA06AB077F557E557D507C44122347123A
:0D5E4400247A8F9E439D80759A0A759BFFFE
:015E5100222E
:031023000262F373
:1062F300C0E0C0F0C083C082C0D075D000C000C071
:0D63030001C002C003C004C005C006C007F1
:10631000C086758600309807C298AF99125229300E
:096320009905C299124CE2D086E5
:10632900D007D006D005D004D003D002D001D000C8
:0B633900D0D0D082D083D0F0D0E03272
:1042BA00253E232E213E1F6C1DB71C1C1A99192D51
:1042CA0017D7169415651447133A123C114D106B03
:1042DA000F960ECD0E0F0D5C0CB20C120B7B0AEC76
:1042EA000A6509E5096B08F9088C082507C30767F9
:1042FA00070F06BC066D062205DB05980558051B47
:10430A0004E104AA04760444041503E803BD0394F3
:10431A00036E03490325030402E402C502A8028DC1
:10432A00027202590241022A021401FF01EB01D76B
:10433A0001C501B401A30193018301750167015904
:10434A00014C014001340129011E0114010A010036
:10435A0000F700EE00E600DE00D600CE00C700C07F
:10436A0000BA00B300AD00A700A2009C009700921B
:10437A00008D008900840080007C00780074007041
:10438A00006D0069006600630060005D005A005716
:10439A0000550052004F004D004B004900460044B2
:0243AA000042CF
:0310000002715525
:1071550075819F007808760008B8A0FAE4900000D1
:10716500F0A3A882A983B8DCF7B907F400025A4254
:102ED400A2AF9253C2AF900234E0FFA3E090032864
:102EE400CFF0A3EFF090022C122751900346122743
:102EF400B79002301227519003791227B790023607
:102F0400E0FFA3E0900367CFF0A3EFF0900220125C
:102F1400275190037E1227B7900224E0FFA3E0908C
:102F24000377CFF0A3EFF090021EE0FEA3E0FFE4EE
:102F3400FCFD9003501227B7851117851218850FD1
:102F4400158510169003621227DC00000000E4903F
:102F54000375F0A3F0A25392AF90034F741EF09048
:102F6400036E745AF0A3740BF0A3740FF09003690A
:102F74001227DCFFFF7748E490036DF0900372049E
:102F8400F090038A7414F090033F743EF0A37480AD
:102F9400F0A3E4F0A37411F09003737406F0A37427
:102FA40022F090038C743CF0900003E02438FE90EF
:102FB4000002E034FF900326F0A3CEF090035A748D
:102FC4000FF0900361740AF0900014E0FFA3E09006
:102FD4000382CFF0A3EFF090034E745AF0E513FB95
:102FE4007A007C117D94FF7E00122514E4FCFD9090
:102FF40003301227B77C0B7DB8AF037E0012251473
:10300400E4FCFD9003561227B7900366743CF090DD
:10301400038B7414F0900334740FF090037D7414D4
:10302400F0900371740AF090032A1227DC00000068
:1030340028900345741EF0900343740BF0A374416D
:10304400F0900354740BF0A37441F0900384E4F003
:10305400A37432F090034AE4F0A37405F090033BA8
:10306400E4F0A37469F0900386E4F0A37464F09030
:10307400034CE4F0A3741EF090033DE4F0A37462E7
:10308400F09003887401F0A37490F090035FE4F06F
:04309400A3744BF0E6
:013098002215
:10634400A2AF9253C2AF900328E0FFA3E0900234BF
:10635400CFF0A3EFF090034612275190022C12279E
:10636400B79003791227519002301227B790036730
:10637400E0FFA3E0900236CFF0A3EFF0A251922207
:10638400A25292209000B9E024FF9221A25392AF2E
:0163940022E6
:06744A005AA569963CC33F
:10409B007F647E00E49002BCF09002BCE0FDC39410
:1040AB000A40030241B9ED25E02402F582E4340015
:1040BB00F583E0FCA3E0D39518EC95175003024170
:1040CB00B09002BCE0705790007AE0FCA3E0FDD307
:1040DB009518EC95175003301906E4FEFF0241B911
:1040EB00C3E5189DFFE5179CFE7C007D0A12283363
:1040FB00EEC0E0EFC0E090007AE0FEA3E0FFC390DB
:10410B000003E09FFF900002E09EFECBEFCBFAE4B2
:10411B00F9F8D0E0FFD0E0FE1226370241B9900249
:10412B00BCE025E02400F582E43400F583E0FEA337
:10413B00E0FFC3E5189FFFE5179EFE7C007D0A128A
:10414B002833ECC0E0EDC0E0EEC0E0EFC0E0900241
:10415B00BCE0FF25E02400F582E43400F583E0FCAD
:10416B00A3E0FDEF25E02402F582E43400F583E0C3
:10417B00FEA3E0C39DFFEE9CFECBEFCBFAE4F9F878
:10418B00D0E0FFD0E0FED0E0FDD0E0FC122637CD32
:10419B00EFCDCCEECC9002BCE075F00AA42DFFE580
:0F41AB00F03CFE80099002BCE004F00240A42228
:103748009002BCEEF0A3EFF09000AAE0F9FDD3EFF1
:103758009DEE9400500302382190036EE0FF900222
:10376800BCE0FCA3E0FDD39FEC94004078ED9464AA
:10377800EC940050709002BCE0FAA3E0FBC37464C0
:103788009BFFE49AFE7C007D0A122514E9FDC3EB39
:103798009DFDEA9CFCD3ED9FEC9E50030238B69049
:1037A80002BCE0FEA3E0FF9000AAF07C007D0A12B4
:1037B80025149003ABEEF0A3EFF09002BCE0FEA35B
:1037C800E0FFE4FD90001AE0F8A3E0F9A3E0FAA313
:1037D800E0FB1225ACE47B64FAF9F8122637900076
:1037E800AB1227B7229002BCE07004A3E0646460C7
:1037F800030238B69000AA7464F09003AB7403F027
:10380800A374E8F090001AE0FCA3E0FDA3E0FEA397
:10381800E0FF9000AB1227B7229000AAE0FD9002CB
:10382800BCE0FEA3E0FFC3ED9FFDE49EFC90034FC8
:10383800E0FBD3ED9BEC9400403F9000AAEFF07CB6
:10384800007D0A1225149003ABEEF0A3EFF090026E
:10385800BCE0FEA3E0FFE4FD90001AE0F8A3E0F965
:10386800A3E0FAA3E0FB1225ACE47B64FAF9F812B2
:1038780026379000AB1227B7229002BCE07002A353
:10388800E0702B9000AA04F09003ABE4F0A3740A54
:10389800F0E47B64FAF9F890001AE0FCA3E0FDA3D9
:0F38A800E0FEA3E0FF1226379000AB1227B722F5
:103A2000122ED412409B9002BAEEF0A3EFF0E47F86
:103A3000E87E03FDFC9000ABE0F8A3E0F9A3E0FA18
:103A4000A3E0FB1225AC90001AE0F8A3E0F9A3E094
:103A5000FAA3E0FB1226379003ABEEF0A3EFF09051
:103A600002BAE0FEA3E0FF1237489000AAE0FF7E12
:103A700000900328EEF0FAA3EFF0FB90001AE0FCB0
:103A8000A3E0FDA3E0FEA3E0FF9003461227B7CF1B
:103A9000EBCF7E00E4FCFD900346E0F8A3E0F9A341
:103AA000E0FAA3E0FB1225ACE47B64FAF9F81226F5
:103AB000379003791227B79000ABE0FCA3E0FDA399
:103AC000E0FEA3E0FF90035B1227B79003371227B5
:103AD000DC000000009003A9E0FFA3E090032ECFDC
:103AE000F0A3EFF0E47830F608F67838F608F678C8
:103AF000341227C3000000009003AF1227DC00003F
:103B00000000E490039FF0A3F09003B5F0A3F090C1
:103B100003ADF0A3F0C252C24EC2509003A8F09081
:103B200003A7F0783AF608F67832F608F69003AB79
:103B3000E0FFA3E09003B3CFF0A3EFF0C251C24D7A
:103B40009003B71227DC00000000E49003A9F0A363
:103B5000F09003911227DC0000000090039A1227D6
:103B6000DC000000009003951227DC00000000E458
:103B700090039EF0900399F0C24F90038D1227DCC2
:083B8000000000001263442262
:10448A0012409B9002BAEEF0A3EFF0900334E0FFE3
:10449A00E4FCFDFE90001AE0F8A3E0F9A3E0FAA319
:1044AA00E0FB1225ACE47B0AFAF9F8122637C8ECCD
:1044BA00C8C9EDC9CAEECACBEFCB90037EE0FCA314
:1044CA00E0FDA3E0FEA3E0FFD31226FA5003024563
:1044DA006090037DE0FF7E009002BAE0FCA3E0FD5D
:1044EA00D39FEC9E4070D3900383E095189003828B
:1044FA00E095174061ED9FFBEC9EFA9003ABE0FE5E
:10450A00A3E0FF7C007D0A122526C3EF9BEE9A509A
:10451A0045900371E0FFC39002BBE09FFF9002BA8F
:10452A00E09400FE7C007D0A1225149003ABEEF0A5
:10453A00A3EFF0E4FD90001AE0F8A3E0F9A3E0FA93
:10454A00A3E0FB1225ACE47BE87A03F9F8122637DC
:07455A009000AB1227B7220D
:101C7A00122ED4900343E0FEA3E0FFD3900378E052
:101C8A009F900377E09E401EE4FFFEFDFC90039ABE
:101C9A00E0F8A3E0F9A3E0FAA3E0FBD31226E440BC
:101CAA0005301802D252C3900383E095189003823C
:101CBA00E095175012900399E004F0E09405400E65
:101CCA007405F0D24E8007C24EE4900399F090005A
:101CDA0028E0FEA3E0FFEE3395E0FDFC90037EE0F2
:101CEA00F8A3E0F9A3E0FAA3E0FBD31226E4500339
:101CFA00021EE2E49003B5F0A3F09003ADF0A3F066
:101D0A0090039EE004F0E0D3940540057405F0D2F8
:101D1A004F9000B9E06010D251E4F09003B7122757
:101D2A00DC00000000C24D900375E0FEA3E0FFEE68
:101D3A003395E0FDFC900281E0F8A3E0F9A3E0FA14
:101D4A00A3E02FFFEA3EFEE93DFDE83CFC9003914B
:101D5A001227B7E4FFFEFDFC900391E0F8A3E0F937
:101D6A00A3E0FAA3E0FBD31226E44021900281E02B
:101D7A00A3E0A3E0FEA3E0FF900376E02FFF900329
:101D8A0075E03EFE783BEF26F618EE36F6C3783B52
:101D9A00E6941018E6940E5003021E2C0874F026DE
:101DAA00F61874F136F690001AE0FCA3E0FDA3E001
:101DBA00FEA3E0FF9000ABE0F8A3E0F9A3E0FAA3EA
:101DCA00E0FBC31226FA50219000ABE0FCA3E0FD31
:101DDA00A3E0FEA3E02401FFE43EFEE43DFDE43C73
:101DEA00FC9000AB1227B7801490001AE0FCA3E025
:101DFA00FDA3E0FEA3E0FF9000AB1227B730518DA0
:101E0A009003B7E0FCA3E0FDA3E0FEA3E02401FFFA
:101E1A00E43EFEE43DFDE43CFC9003B71227B70222
:101E2A001D97900343E0FEA3E0FFD3900378E09F61
:101E3A00900377E09E404490006AE0FEA3E0FFEE44
:101E4A003395E0FDFC900281E0F8A3E0F9A3E0FA03
:101E5A00A3E0FBC31226E45022C3900069E0951860
:101E6A00900068E09517501390006CE0FF9003A86B
:101E7A00E004F0C39F4004EFF0D25290006AE0FE03
:101E8A00A3E0FFEE3395E0FDFC900281E0F8A3E0C9
:101E9A00F9A3E0FAA3E0FBC31226E45035900350FD
:101EAA00E0FCA3E0FDA3E0FEA3E0FF900330E0F82E
:101EBA00A3E0F9A3E0FAA3E0FBC31226FA501390B9
:101ECA000366E0FF9003A7E004F0C39F4004EFF02D
:101EDA00D25012448A022220900028E0FEA3E0FF9A
:101EEA00C3E49FFFE49EFE3395E0FDFC90037EE091
:101EFA00F8A3E0F9A3E0FAA3E0FBC31226E4400347
:101F0A000220D7E49003A8F09003A7F0C250C2526F
:101F1A009003ADF0A3F09003B6F090039EF0C24F89
:101F2A00900362E0FCA3E0FDA3E0FEA3E0FF9002C1
:101F3A0081E0F8A3E0F9A3E0FAA3E02FFBEA3EFA76
:101F4A00E93DF9E83CF8900375E0FEA3E0FFEE33C3
:101F5A0095E0FDFCEB2FFFEA3EFEE93DFDE83CFC87
:101F6A009003911227B7900391E0FCA3E0FDA3E050
:101F7A00FEA3E0FFEC33500AC37833E69FF618E677
:101F8A009EF6C37833E6941018E6940E50030220A6
:101F9A006CC37833E6941018E6940E40670874F020
:101FAA0026F61874F136F69000B3E0FCA3E0FDA320
:101FBA00E0FEA3E02401FFE43EFEE43DFDE43CFC38
:101FCA009000B31227B7E47F01FEFDFC9000ABE05E
:101FDA00F8A3E0F9A3E0FAA3E0FBD31226FA40B192
:101FEA009000ABE0FCA3E0FDA3E0FEA3E024FFFF2A
:101FFA00EE34FFFEED34FFFDEC34FFFC9000AB1233
:10200A0027B7808D90001EE0FCA3E0FDA3E0FEA3AD
:10201A00E0FF9000B3E0F8A3E0F9A3E0FAA3E0FB45
:10202A00C31226FA403C9000B3E0FCA3E0FDA3E013
:10203A00FEA3E0FF90001EE0F8A3E0F9A3E0FAA3F4
:10204A00E0FBEF9BFFEE9AFEED99FDEC98FC900009
:10205A00B31227B7900023E004F07006900022E044
:10206A0004F0900354E0FEA3E0FFD3900378E09FCE
:10207A00900377E09E50030222209000AFE0FCA379
:10208A00E0FDA3E0FEA3E0FF900281E0F8A3E0F9FF
:10209A00A3E0FAA3E0FBD31226E45003022220D3E2
:1020AA0090007BE0951690007AE095155003022285
:1020BA002090007CE0FF9003B5E004F09F500302FB
:1020CA002220EFF09000B97401F0022220900375EB
:1020DA00E0FAA3E0FBFFCEEACEEE3395E0FDFC3357
:1020EA0040030221CAC37833E69BFF18E69AFEF63C
:1020FA0008EFF6C39410EE940E50030221CA74F04E
:10210A0026F61874F136F69000B3E0FCA3E0FDA3BE
:10211A00E0FEA3E02401FFE43EFEE43DFDE43CFCD6
:10212A009000B31227B7E47F01FEFDFC9000ABE0FC
:10213A00F8A3E0F9A3E0FAA3E0FBD31226FA4022BF
:10214A009000ABE0FCA3E0FDA3E0FEA3E024FFFFC8
:10215A00EE34FFFEED34FFFDEC34FFFC9000AB12D1
:10216A0027B790001EE0FCA3E0FDA3E0FEA3E0FF7A
:10217A009000B3E0F8A3E0F9A3E0FAA3E0FBC312EE
:10218A0026FA403C9000B3E0FCA3E0FDA3E0FEA3E6
:10219A00E0FF90001EE0F8A3E0F9A3E0FAA3E0FB59
:1021AA00EF9BFFEE9AFEED99FDEC98FC9000B312BE
:1021BA0027B7900023E004F07006900022E004F0B4
:1021CA0090038CE0FF9003ADE475F00112257BFCCF
:1021DA00C3E5F09FEC9400403A900354E0FEA3E07C
:1021EA00FFD3900378E09F900377E09E4025D39039
:1021FA00007BE0951690007AE09515401690007CD9
:10220A00E0FF9003B6E004F09F4008EFF09000B9B9
:10221A007401F0122860E47FE87E03FDFC9000ABB5
:10222A00E0F8A3E0F9A3E0FAA3E0FB1225AC9000E2
:10223A001AE0F8A3E0F9A3E0FAA3E0FB122637902C
:10224A0003ABEEF0A3EFF0900028E0FEA3E0FFC39B
:10225A00E49FFFE49EFE3395E0FDFC90037EE0F8E8
:10226A00A3E0F9A3E0FAA3E0FBC31226E4400C20A2
:10227A001509201A06201B03301C02C251121056DF
:10228A009000AAE0FF7E00900328EEF0FAA3EFF098
:10229A00FB90001AE0FCA3E0FDA3E0FEA3E0FF90A0
:1022AA0003461227B7CFEBCF7E00E4FCFD9003462E
:1022BA00E0F8A3E0F9A3E0FAA3E0FB1225ACE47B83
:1022CA0064FAF9F81226379003791227B790002298
:1022DA00E0FFA3E0900367CFF0A3EFF09003ABE039
:1022EA00FFA3E09003B3CFF0A3EFF0900391E0FCDB
:1022FA00A3E0FDA3E0FEA3E0FF90039A1227B790A4
:10230A0000ABE0FCA3E0FDA3E0FEA3E0FF90035BCB
:10231A001227B79003AFE0FCA3E0FDA3E0FEA3E021
:10232A00FF9003371227B79003A9E0FFA3E09003B9
:0A233A002ECFF0A3EFF0126344224F
:106EA500122ED490038D12277690032AE0F8A3E0E2
:106EB500F9A3E0FAA3E0FBC31226FA501490032AC3
:106EC500E0FCA3E0FDA3E0FEA3E0FF90038D122705
:056ED500B71263442226
:102AB8009005F7E4F0A37464F0122ED412409B90B2
:102AC80005F7EEF0A3EFF04E702E9000AA04F090F8
:102AD80003ABE4F0A3740AF0E47B64FAF9F890001D
:102AE8001AE0FCA3E0FDA3E0FEA3E0FF1226379066
:102AF80000AB1227B7022BC290032AE0FCA3E0FD2B
:102B0800A3E0FEA3E0FF90038DE0F8A3E0F9A3E0C3
:102B1800FAA3E0FBC31226FA400E9005F7E0FEA3E5
:102B2800E0FF123748022BC2E47F64FEFDFC9000F0
:102B38001AE0F8A3E0F9A3E0FAA3E0FB1225AC90B1
:102B480000ABE0F8A3E0F9A3E0FAA3E0FB12263714
:102B5800C8ECC8C9EDC9CAEECACBEFCB90034FE0A9
:102B6800FF9005F8E02FFF9005F7E03400FEE4FC45
:102B7800FDD31226FA40439005F7E0FAA3E0FB7C68
:102B8800007D0AFFCEEACE1225149003ABEEF0A327
:102B9800EFF0CFEBCFCEEACEE4FD90001AE0F8A339
:102BA800E0F9A3E0FAA3E0FB1225ACE47B64FAF9B0
:102BB800F81226379000AB1227B7E47830F608F6FB
:102BC8007838F608F678341227C30000000090031E
:102BD800AF1227DC00000000E490039FF0A3F09000
:102BE80003B5F0A3F09003ADF0A3F0C252C24EC2F9
:102BF800509003A8F09003A7F0783AF608F67832D8
:102C0800F608F69003ABE0FFA3E09003B3CFF0A380
:102C1800EFF0C251C24D9003B71227DC000000004C
:102C2800E49003A9F0A3F09003911227DC000000C0
:102C38000090039A1227DC000000009003951227E9
:102C4800DC00000000E490039EF0900399F0C24F6E
:102C580090038D1227DC000000009000AAE0FF7EA0
:102C680000900328EEF0FAA3EFF0FB90001AE0FCC6
:102C7800A3E0FDA3E0FEA3E0FF9003461227B7CF31
:102C8800EBCF7E00E4FCFD900346E0F8A3E0F9A357
:102C9800E0FAA3E0FB1225ACE47B64FAF9F812260B
:102CA800379003791227B79000ABE0FCA3E0FDA3AF
:102CB800E0FEA3E0FF90035B1227B79003371227CB
:102CC800DC00000000E490032EF0A3F0126344221D
:10286000305109305206C251D24D802130521E9053
:1028700003AB7403F0A374E8F090001AE0FCA3E04B
:10288000FDA3E0FEA3E0FF9000AB1227B7304D039D
:102890000229109000B7E0FCA3E0FD900022E0FECA
:1028A000A3E0FFC39DFDEE9CFCC3900360E09D9000
:1028B000035FE09C4003022AB7205203022AB712AA
:1028C0005F6FE4FCFDFE90001AE0F8A3E0F9A3E0DE
:1028D000FAA3E0FB1225ACECC0E0EDC0E0EEC0E0F6
:1028E000EFC0E09000B7E0FEA3E0FF125F6FCBEF18
:1028F000CBE4FAF9F8D0E0FFD0E0FED0E0FDD0E084
:10290000FC1226379003B71227B7022A6C022A6CF2
:10291000C24DE47F32FEFDFC900016E0F8A3E0F922
:10292000A3E0FAA3E0FB1225ACE47B64FAF9F81209
:1029300026379002BA1227B79002BAE0FCA3E0FD56
:10294000A3E0FEA3E0FF9003B7E0F8A3E0F9A3E063
:10295000FAA3E02FFFEA3EFEE93DFDE83CFC9000D3
:1029600016E0F8A3E0F9A3E0FAA3E0FBC31226FA0D
:102970004003022AB7900345E0FFE4FCFDFE90000F
:102980001AE0F8A3E0F9A3E0FAA3E0FB1225ACE417
:102990007B64FAF9F81226379002BA1227B7900230
:1029A000BAE0FCA3E0FDA3E0FEA3E0FF90001AE084
:1029B000F8A3E0F9A3E0FAA3E02FFFEA3EFEE93D29
:1029C000FDE83CFC9003B7E0F8A3E0F9A3E0FAA32C
:1029D000E0FBD31226FA402E9002BAE0FCA3E0FD01
:1029E000A3E0FEA3E0FF90001AE0F8A3E0F9A3E063
:1029F000FAA3E02FFFEA3EFEE93DFDE83CFC900330
:102A0000B71227B780669002BAE0FCA3E0FDA3E00E
:102A1000FEA3E0FF9003B7E0F8A3E0F9A3E0FAA378
:102A2000E02FFFEA3EFEE93DFDE83CFC90001AE0A5
:102A3000F8A3E0F9A3E0FAA3E0FBD31226FA402CB6
:102A40009002BAE0F8A3E0F9A3E0FAA3E0FB90005B
:102A50001AE0FCA3E0FDA3E0FEA3E09BFFEE9AFEDC
:102A6000ED99FDEC98FC9003B71227B79003B7E0FF
:102A7000FCA3E0FDA3E0FEA3E0FF90001A1227B73D
:102A80009003AB7403F0A374E8F090001AE0FCA389
:102A9000E0FDA3E0FEA3E0FF9000AB1227B790009B
:102AA00022E0FFA3E09000B7CFF0A3EFF09003B7D0
:082AB0001227DC0000000022E7
:105F6F00C3900389E09F900388E09E500479558089
:105F7F0048C3900387E09F900386E09E50169003DE
:105F8F004CE0FCA3E0FD12252690033DE0A3E0C307
:105F9F009FF98025C3900385E09F900384E09E5076
:105FAF001690034AE0FCA3E0FD12252690033BE088
:0D5FBF00A3E0C39FF980027964CFE9CF22EF
:10105600E49002BAF0A3F0FFA3F0A3F0A3F090038C
:10106600A1E0645A6028A2AF9253C2AF75A701E40B
:10107600EF90124093FE74A12FF582E43403F583BA
:10108600EEF00FEFB406E9E4F5A7A25392AF900392
:10109600A6E064C36003021C48FF74A12FF582E436
:1010A6003403F583E0FEEF90744A936E6003021CEE
:1010B600480FEFB406E48003021C48900028E0FEC7
:1010C600A3E0FFEE3395E0FDFC90037EE0F8A3E09D
:1010D600F9A3E0FAA3E0FBD31226E450030214F1CD
:1010E600204F030214F1E47830F608F67838F60853
:1010F600F69000AAE0D394634003021C48C3900311
:1011060083E09518900382E09517401E90034EE009
:10111600FF7E007C007D0A122514D39003ACE09F6D
:101126009003ABE09E50030213C9304E5A90034E13
:10113600E0FBFF7E007C007D0A1225149003ACE0E4
:101146002496FD9003ABE03400FCC3ED9FEC9E506B
:1011560036EBFF7E007C007D0A122514EEF0A3EF2D
:10116600F0CFEBCFE4FDFE90001AE0F8A3E0F9A380
:10117600E0FAA3E0FB1225ACE47B64FAF9F8122648
:10118600379000AB1227B7900350E0FCA3E0FDA315
:10119600E0FEA3E0FF900330E0F8A3E0F9A3E0FA55
:1011A600A3E0FBD31226FA5003021230900350E05C
:1011B600F8A3E0F9A3E0FAA3E0FB900330E0FCA378
:1011C600E0FDA3E0FEA3E09BFBEE9AFAED99F9ECB5
:1011D60098F890038AE0FFE4FCFDFE1225ACE47B60
:1011E6000AFAF9F81225ACEEC0E0EFC0E090001460
:1011F600E0FEA3E0FFC3900069E09FFF900068E077
:101206009EFECBEFCBFAE4F9F8D0E0FFD0E0FE1279
:101216002637EFC0E0AF13CBEFCBE4FAF9F8D0E016
:10122600FF1226379003951227B7C3900063E09507
:1012360018FF900062E09517FE90038AE0FD7C009F
:10124600122833E47B0AFAF9F81225ACEEC0E0EF77
:10125600C0E0900014E0FEA3E0FFC3900069E09FA9
:10126600FF900068E09EFECBEFCBFAE4F9F8D0E001
:10127600FFD0E0FE1226379002BF1227B7900395E3
:10128600E0FCA3E0FDA3E0FEA3E0FF9002BFE0F8D0
:10129600A3E0F9A3E0FAA3E0FBC31226FA501490E8
:1012A60002BFE0FCA3E0FDA3E0FEA3E0FF900395F0
:1012B6001227B7E47F24FEFDFC90001AE0F8A3E0B5
:1012C600F9A3E0FAA3E0FB1225AC900395E0F8A39E
:1012D600E0F9A3E0FAA3E0FB1225ACEEC0E0EFC014
:1012E600E09000AAE0FFC374659FFFE49400FECB84
:1012F600EFCBFAE4F9F8D0E0FFD0E0FE122637E4AF
:101306007B0AFAF9F81226379003951227B7900050
:101316006AE0FEA3E0FFEE3395E0FDFC900391E06A
:10132600F8A3E0F9A3E0FAA3E0FBD31226E4406CAD
:10133600900391E0FCA3E0FDA3E0FEA3E0FFC8EC70
:10134600C8A3E0FCA3E0FDA3E0FEA3E0FF1226375E
:10135600ECC0E0EDC0E0EEC0E0EFC0E090006AE077
:10136600FEA3E0FFFBCAEECAEA3395E0F9F8900364
:1013760091E0FCA3E0FDA3E0FEA3E0C39BFFEE9A91
:10138600FEED99FDEC98FCD0E0FBD0E0FAD0E0F958
:10139600D0E0F81225AC9003951227B7900063E0D1
:1013A60024FFFF900062E034FFFEC3E5189FE517B7
:1013B6009E50030214839003951227DC0000000060
:1013C6000214839003ABE0FEA3E0FF7C007D0A12CB
:1013D6002526EF2401FFE43EFE9000AAE0FB7A00FA
:1013E600C39FEA9E503C9003ABE0FEA3E0FF7C0067
:1013F6007D0A122526EB2401FDEA33FCD3ED9FEC92
:101406009E401FE47F24FEFDFC90001AE0F8A3E056
:10141600F9A3E0FAA3E0FB1225AC9003951227B7D7
:10142600805B9000ABE0F8A3E0F9A3E0FAA3E0FB51
:1014360090001AE0FCA3E0FDA3E0FEA3E0C39BFF3F
:10144600EE9AFEED99FDEC98FCE47B107A0EF9F825
:101456001225ACEEC0E0EFC0E09000AAE0FFC37436
:10146600649FFFE49400FECBEFCBFAE4F9F8D0E0FA
:10147600FFD0E0FE1226379003951227B79003910E
:10148600E0FCA3E0FDA3E0FEA3E0FFFBCAEECAC9B1
:10149600EDC9C8ECC8A3E0FCA3E0FDA3E0FEA3E011
:1014A600FF1226379002BDEEF0A3EFF02050033076
:1014B600520D90038BE0FF9002BDE4F0A3EFF09095
:1014C60003A9E475F00112257BFEC39002BEE095E8
:1014D600F09002BDE09E4003021C489000AAE00482
:1014E600F0E49003A9F0A3F0021C48900028E0FE67
:1014F600A3E0FFC3E49FFFE49EFE3395E0FDFC906E
:10150600037EE0F8A3E0F9A3E0FAA3E0FBC312260A
:10151600E44003021BE89000AAE094015003021C79
:1015260048900326E0FEA3E0FFAD137C00122833AB
:10153600900350E0F8A3E0F9A3E0FAA3E0FBC3129E
:1015460026FA402DD390007BE0951690007AE09520
:1015560015501E90035AE0FF7E007C007D0A12257E
:1015660014C39003ACE09F9003ABE09E40030218C7
:101576000B90036FE0FEA3E0FFD3900378E09F900B
:101586000377E09E500302180B900369E0FCA3E08A
:10159600FDA3E0FEA3E0FF90037EE0F8A3E0F9A33D
:1015A600E0FAA3E0FBD31226E4500302180B7839C5
:1015B600E61846700302180B90039AE0FCA3E0FDC0
:1015C600A3E0FEA3E024D0FFEE3407FEE43DFDE4F5
:1015D6003CFC900391E0F8A3E0F9A3E0FAA3E0FB5A
:1015E600C31226E4400302180B90039AE0FCA3E022
:1015F600FDA3E0FEA3E02430FFEE34F8FEED34FF59
:10160600FDEC34FFFC900391E0F8A3E0A3E0A3E037
:10161600D31226E4500302180B900361E07E0025E6
:1016260016FFEE3515FEC3EF783996EE1896400391
:101636000217FA90039FE0FEA3E0FF9400EE9400E9
:1016460050030217FAEF9401EE9400500890039F9E
:10165600E4F0A304F0900350E0FCA3E0FDA3E0FE59
:10166600A3E0FF783412275DD31226FA500302173F
:1016760013900356E0F8A3E0F9A3E0FAA3E0FB9089
:101686000350E0FCA3E0FDA3E0FEA3E09BFBEE9A83
:10169600FAED99F9EC98F890039FE0FEA3E0FFE4D9
:1016A600FCFD1225ACECC0E0EDC0E0EEC0E0EFC002
:1016B600E0900350E0F8A3E0F9A3E0FAA3E0FBE82A
:1016C600C0E07834122745D0E0F8C3EF9BFBEE9AD2
:1016D600FAED99F9EC98F8D0E0FFD0E0FED0E0FD05
:1016E600D0E0FC122637EEC0E0EFC0E09000AAE0A2
:1016F60024FFFFE434FFFECBEFCBFAE4F9F8D0E0A9
:10170600FFD0E0FE1226379003951227B79000749B
:10171600E0FEA3E0FFC3E5169FFFE5159EFE9003DE
:101726009FE0FCA3E0FD122833EEC0E0EFC0E0C36B
:101736007839E69516FF18E69515FECBEFCBFAE459
:10174600F9F8D0E0FFD0E0FE122637EEC0E0EFC099
:10175600E09000AAE024FFFFE434FFFECBEFCBFAD3
:10176600E4F9F8D0E0FFD0E0FE1226379002BF126F
:1017760027B7900395E0FCA3E0FDA3E0FEA3E0FFFE
:101786009002BFE0F8A3E0F9A3E0FAA3E0FBC312DE
:1017960026FA50149002BFE0FCA3E0FDA3E0FEA3EE
:1017A600E0FF9003951227B77838A61508A616907D
:1017B6000350E0FCA3E0FDA3E0FEA3E0FF783412B3
:1017C60027ABE490039FF0A3F0900395E0F8A3E025
:1017D600F9A3E0FAA3E0FB900391E0FCA3E0FDA3EC
:1017E600E0FEA3E0FF1226D61225AC900395122741
:1017F600B7021B769003A0E004F0700690039FE00A
:1018060004F0021B767838A61508A616900350E059
:10181600FCA3E0FDA3E0FEA3E0FF78341227ABE4CF
:1018260090039FF0A3F090036FE0FEA3E0FFC39048
:101836000378E09F900377E09E4021900369E0FCE7
:10184600A3E0FDA3E0FEA3E0FF90037EE0F8A3E0A3
:10185600F9A3E0FAA3E0FB1226E4501D90001AE07B
:10186600FCA3E0FDA3E0FEA3E0FF9003AF1227B7C1
:10187600E47830F608F60219FA7830E6FE08E6FF54
:101886002414FDE43EFC900377E0FAA3E0FBD39D2D
:10189600EA9C5011EB2414FDE43AFCD3EF9DEE9C38
:1018A60050030219FA900377E0FEA3E0FF7830EECA
:1018B600F608EFF62487FFEE34F59002BAF0A3EFB0
:1018C600F0900341E0FEA3E0FFFBCAEECAE4F9F89C
:1018D6009002BAE0FEA3E0FFEE3395E0FDFC122590
:1018E600ACC8ECC8C9EDC9CAEECACBEFCB90033F72
:1018F600E0FEA3E0FFE4C3EF9BFBEE9AFAE499F95E
:10190600E498F89002BAE0FEA3E0FFEE3395E0FD1E
:10191600FC1225ACE47B107A27F9F8126ADCC8ECD5
:10192600C8C9EDC9CAEECACBEFCB900373E0FEA3DC
:10193600E0FFE4FCFDEB2FFFEA3EFEED39FDEC385F
:10194600FC90001AE0F8A3E0F9A3E0FAA3E0FB128A
:1019560025ACE47BD07A07F9F81226379003AF124C
:1019660027B790001AE0FCA3E0FDA3E0FEA3E0FF8A
:101976009003AFE0F8A3E0F9A3E0FAA3E0FBD312EB
:1019860026FA401690001AE0FCA3E0FDA3E0FEA3B1
:10199600E0FF9003AF1227B7805AE47F06FEFDFCF6
:1019A60090001AE0F8A3E0F9A3E0FAA3E0FB122501
:1019B600ACE47B0AFAF9F81226379003AFE0F8A3F5
:1019C600E0F9A3E0FAA3E0FBC31226FA5026E47F6F
:1019D60006FEFDFC90001AE0F8A3E0F9A3E0FAA3E6
:1019E600E0FB1225ACE47B0AFAF9F81226379003DD
:1019F600AF1227B79003AFE0F8A3E0F9A3E0FAA38C
:101A0600E0FB90001AE0FCA3E0FDA3E0FEA3E0C328
:101A16009BFFEE9AFEED99FDEC98FCE47B0DFAF93E
:101A2600F81225ACE47B0AFAF9F81226379000ABD7
:101A3600E0F8A3E0F9A3E0FAA3E0FBC31226FA500C
:101A460020E47F24FEFDFC90001AE0F8A3E0F9A351
:101A5600E0FAA3E0FB1225AC9003951227B7021B10
:101A6600769000ABE0FCA3E0FDA3E0FEA3E0FF90D0
:101A760003AFE0F8A3E0F9A3E0FAA3E02FFFEA3E04
:101A8600FEE93DFDE83CFC90001AE0F8A3E0F9A36E
:101A9600E0FAA3E0FBC3EF9BFFEE9AFEED99FDECA7
:101AA60098FCE47B64FAF9F81225AC9003AFE0F8F1
:101AB600A3E0F9A3E0FAA3E0FB1226379002BCEFFD
:101AC600F02401FFE433FE9000AAE0FDC39FEE641C
:101AD60080F87480985035ED2401FFE433FE9002BF
:101AE600BCE0FDD3EF9D7480F86E98401FE47F2420
:101AF600FEFDFC9003AFE0F8A3E0F9A3E0FAA3E053
:101B0600FB1225AC9003951227B780649000ABE0DA
:101B1600FCA3E0FDA3E0FEA3E0FF9003AFE0F8A383
:101B2600E0F9A3E0FAA3E02FFFEA3EFEE93DFDE877
:101B36003CFC90001AE0F8A3E0F9A3E0FAA3E0FB6E
:101B4600C3EF9BFFEE9AFEED99FDEC98FCE47B104B
:101B56007A0EF9F81225ACEFC0E09000AAE0FFFB80
:101B6600E4FAF9F8D0E0FF1226379003951227B76A
:101B7600900391E0FCA3E0FDA3E0FEA3E0FF1226A4
:101B8600D6CBEFCBCAEECAC9EDC9C8ECC8A3E0FCF8
:101B9600A3E0FDA3E0FEA3E0FF1226379002BDEE10
:101BA600F0A3EFF09003A9E475F00112257BFCD3B6
:101BB600E5F09FEC9E400D9000AAE014F0E490033F
:101BC600A9F0A3F030197B900372E0FF9000AAE021
:101BD600D39F506E90036DE060689000AA7401F088
:101BE6008060E47838F608F678341227C3000000DF
:101BF60000E47830F608F69000AAE0D3940140425B
:101C0600900375E0FEA3E0FFEE3395E0FDFC335054
:101C1600319003ABE0FEA3E0FF7C007D0A1225268F
:101C2600CAEECACBEFCB9003B3E0FEA3E0FF7C0085
:101C36007D0A122526D3EF9BEE9A40069000AAE075
:101C460014F0E4FFFEFDFC90039AE0F8A3E0F9A38C
:101C5600E0FAA3E0FBD31226E44009301806900010
:101C6600AA7464F09002BDE0FFA3E0900335CFF0C4
:041C7600A3EFF022C6
:1071EC00304C19204306204403304510C24CC24396
:0D71FC00C244C245C2AF1273611200A62248
:10000000020D7A021003000000000002100B000035
:10001000000000021013000000000002101B00008E
:10002000000000021023000000000002102B00005E
:10003000000000021033000000000002103B00002E
:10004000000000021043000000000002104B0000FE
:10005000000000021053000000000002105B0000CE
:10006000000000021063000000000002106B00009E
:10007000000000021073000000000002107B00006E
:10008000000000021083000000000002108B00003E
:10009000000000021093000000000002109B00000E
:1000A0000000000210A3E4F526F525F524F523F55C
:1000B00030F52FF52EF52DF52C120D5E209803024C
:1000C000018E7400252BF582E43402F583E599F066
:1000D000052BE52BC3948C4003E4F52BE52BB401F1
:1000E0000D900200E0645A700302018C806BE52BD6
:1000F000B40214900201E064A56002805CE4F53172
:10010000F532F52202018C900202E0FF7E00240904
:10011000FDEE33FCAB2B7A00C3EB9DEC6480F874EE
:1001200080985062EF2407FFEE33FED3EB9FEE641E
:1001300080F8748098501574FF252BF582E4340103
:10014000F583E02532F532E43531F531E52BB405A0
:100150000D900204E064076033E4F52B802EE52B5C
:1001600064067028900205E0FF6406601FEF6407D4
:10017000601AEF64086015EF64096010EF640A60AC
:100180000B432230800653B1F8120A9DC298309971
:100190004453B1F8900202E02408FFE433FEC3E5C3
:1001A0002B9FEE6480F87480984013E4F586D29C0F
:1001B000F52B900200F0A3F0A3F0D2028015052BDE
:1001C000E4F586C29C7400252BF582E43402F583A5
:1001D000E0F599C299E52C640A60030200BC53B1B2
:1001E000F82002030200BCC202F52C12000002003B
:1001F000BCC200900206E0FFC395214014E5212413
:1002000004FDE433FCD3EF9DEC6480F874809840E7
:100210000A900206E060047405F022900206E0F500
:1002200021E4F0900202E070152526F526E525343C
:1002300002F525E43524F524E43523F52322E521D0
:100240005403F50AE4F508F509900202E0FD7C008C
:10025000C3E5099DE5089C503274072509F582E441
:100260003402F583E0FBAF0A7E00120638E5092F61
:10027000FFE5083EFE74002FF58274003EF583EB27
:10028000F00509E50970C2050880BEE50A6403604F
:100290000302044F751D551208955003020386E4AE
:1002A000FF7E02FDFCAB26AA25A924A8231207186D
:1002B000401AE5269400F526E5259402F525E52467
:1002C0009400F524E5239400F5238009E4F526F550
:1002D00025F524F523E4F50F30015E2526F50EE51E
:1002E000253410F50DE43524F50CE43523F50BE445
:1002F000252AFFE529340CFEE43528FDE43527FCEA
:10030000AB0EAA0DA90CA80BC31207184040E42598
:100310002AFBE529340CFAE43528F9E43527F8C33B
:10032000E50E9BF50EE50D9AF50DE50C99F50CE53E
:100330000B98F50B750F018015E42526F50EE525C4
:100340003484F50DE43524F50CE43523F50B751DE7
:1003500055AF0EAE0DAD0CAC0B850F15120B7EAF6D
:100360000EAE0DAD0CAC0B850F15120C8C500E1291
:10037000089540129002067403F002044C900206A5
:100380007402F002044CE4F50A75F004E50AA424B2
:1003900002F582E5F03400F583E0FFE4FCFDFE7831
:1003A0001012073CC004C005C006C00775F004E584
:1003B0000AA42403F582E5F03400F583E0FFE4FCB1
:1003C000FDFE781812073CD003D002D001D000EF18
:1003D0004BFFEE4AFEED49FDEC48FCC004C005C0F1
:1003E00006C00775F004E50AA42401F582E5F0349F
:1003F00000F583E0FFE4FCFDFE780812073CD00323
:10040000D002D001D000EF4BFBEE4AFAED49F9ECF7
:1004100048F875F004E50AA42400F582E5F03400FC
:10042000F583E0FFEB4FFFEAFEE9FDE8FCE5302F46
:10043000F530E52F3EF52FE52E3DF52EE52D3CF56B
:100440002D050AE50A64806003020389E4F51D2294
:10045000E4F526F525F524F523F530F52FF52EF5F1
:100460002DF52AF529F528F527900209E0FFE4FC8F
:10047000FDFE781012073CC004C005C006C007A3EB
:10048000E0FFE4FCFDFE781812073CD003D002D058
:1004900001D000EF4BFFEE4AFEED49FDEC48FCC0F9
:1004A00004C005C006C007900208E0FFE4FCFDFEA2
:1004B000780812073CD003D002D001D000EF4BFBEC
:1004C000EE4AFAED49F9EC48F8900207E0FFEB4FED
:1004D000F52AEAF529E9F528E8F527200006900233
:1004E00006740AF0E4FF7E78FDFCAB2AAA29A9284D
:1004F000A827D312071840052001028017E4FF7EC9
:10050000ECFDFCAB2AAA29A928A827D3120718407A
:100510000A3001079002067401F022E4900206F00E
:10052000F521751D55F515FF7E0EFDFC120B7EE4C1
:10053000F515FF7E0EFDFC120C8C502B30012E7534
:100540001BA5E4F51C7FFF7E0FFDFC120B15E4F5E7
:100550001B7FFF7E0FFDFC120D94EF64A5600E90D3
:1005600002067403F080069002067402F0E4F51DA2
:10057000900206E06003020631FB7A02F9F8AF2A26
:10058000AE29AD28AC271206868F09E4F508E508E8
:10059000C395094003020637E4F50A300107F50E5A
:1005A000750D108006E4F50E750D84F50CF50BE560
:1005B0000825E0FEE4FCFD250EF50EE50D3EF50DEB
:1005C000ED350CF50CEC350BF50B300135E5092458
:1005D000FEFBE434FFFAED34FFF9EC34FFF8AF082A
:1005E000E4FED3120718501A750A01E5082402FF29
:1005F000C3EF9509FFEF25E0FEE4F50E8E0DF50C37
:10060000F50B751D55AF0EAE0DAD0CAC0B850A1577
:10061000120B7EAF0EAE0DAD0CAC0B850A15120C95
:100620008C40069002067402F0E4F51D05080205F0
:100630008E9002067405F022EF8DF0A4A8F0CF8C06
:10064000F0A428CE8DF0A42EFE2275F0087582004D
:10065000EF2FFFEE33FECD33CDCC33CCC58233C587
:10066000829BED9AEC99E58298400CF582EE9BFE18
:10067000ED9AFDEC99FC0FD5F0D6E4CEFBE4CDFA73
:10068000E4CCF9A88222B800C1B90059BA002DEC17
:100690008BF084CFCECDFCE5F0CBF97818EF2FFFAF
:1006A000EE33FEED33FDEC33FCEB33FB10D7039957
:1006B0004004EB99FB0FD8E5E4F9FA227818EF2F04
:1006C000FFEE33FEED33FDEC33FCC933C910D70523
:1006D0009BE99A4007EC9BFCE99AF90FD8E0E4C942
:1006E000FAE4CCFB2275F010EF2FFFEE33FEED3372
:1006F000FDCC33CCC833C810D7079BEC9AE899409F
:100700000AED9BFDEC9AFCE899F80FD5F0DAE4CD00
:10071000FBE4CCFAE4C8F922EB9FF5F0EA9E42F044
:10072000E99D42F0E89C45F022E8600FECC313FC21
:10073000ED13FDEE13FEEF13FFD8F122E8600FEF8B
:10074000C333FFEE33FEED33FDEC33FCD8F122EC86
:100750008EF0A4CCC5F0CCCDF8EFA4CEC5F02DFD25
:10076000E43CFCE8A42EC8C5F03DFDE43CFCEFA44D
:10077000FFE5F028FEE43DFDE43CFC22E4F50853EF
:10078000B1F8E508C3943A501FE4F50AAF08FE7CBF
:1007900002FD12074FE42FF510EE3410F50FE43D83
:1007A000F50EE43CF50D8021750A01AF087E007C52
:1007B000027D0012074FE42FF510EE348CF50FED9B
:1007C00034FFF50EEC34FFF50D751D55AF10AE0F6F
:1007D000AD0EAC0D850A15120B7EAF10AE0FAD0E2F
:1007E000AC0D850A15120C8C4003020883E4F50B4E
:1007F000F50CAE0BAF0CE4FCFDFB7A02F9F8D3125A
:1008000007185003020886AF087E007C027D0012A4
:10081000074FA804A905AA06AB07E4250CFFE50BC2
:100820003484FEE433FDE433FCEB2FFFEA3EFEE9C3
:100830003DFDE83CFCE4F51B120D948F09E50C2509
:1008400010FFE50B350FFEE4350EFDE4350DFC859C
:10085000091B850A1C120B15E50C2510FFE50B354D
:100860000FFEE4350EFDE4350DFC850A1B120D94D8
:10087000EF650960037F0222050CE50C7002050B91
:100880000207F27F01220508E508C3943C500302E9
:10089000077F7F0022D203E4F510F511AE10AF11EF
:1008A000E4FCFDFB7A02F9F8D312071850030209A1
:1008B0008CE4F51630015E2526F515E5253410F596
:1008C00014E43524F513E43523F512E4252AFFE575
:1008D00029340CFEE43528FDE43527FCAB15AA14B9
:1008E000A913A812C31207184040E4252AFBE529E2
:1008F000340CFAE43528F9E43527F8C3E5159BF5FF
:1009000015E5149AF514E51399F513E51298F51207
:100910007516018015E42526F515E5253484F514B2
:10092000E43524F513E43523F512AF15AE14AD13F9
:10093000AC1274002511F58274003510F583E0F5D2
:100940001B85161C120B15AF15AE14AD13AC12851A
:10095000161B120D9474002511F58274003510F5E4
:1009600083E06F6004C2038023E5262401F526E4BA
:100970003525F525E43524F524E43523F523051143
:10098000E511600302089C051002089CA203227E68
:10099000007D007C00900209E0FFE4781012073C23
:1009A000C004C005C006C007A3E0FFE4FCFDFE785C
:1009B0001812073CD003D002D001D000EF4BFFEE5D
:1009C0004AFEED49FDEC48FCC004C005C006C00766
:1009D000900208E0FFE4FCFDFE780812073CD0031B
:1009E000D002D001D000EF4BFBEE4AFAED49F9EC12
:1009F00048F8900207E0FFEB4FFFEAFEE9FDE8FC54
:100A0000AB30AA2FA92EA82DC31207186007900299
:100A1000067408F022E4900206F022E4F508F509D5
:100A2000900202F0900205740BF0900203E0FFA325
:100A3000E0900203F0A3EFF07F02900202E0FE24B8
:100A400007FDE433FCEFC39DEC6480F8748098509C
:100A50001774002FF582E43402F583E02509F509C7
:100A6000E43508F5080F80D274072EF582E43402CD
:100A7000F583E509F0E508FF900202E02408F5821D
:100A8000E43402F583EFF0C202E4F586C29C740000
:100A9000252BF582E43402F583E0F59922E4F52B69
:100AA000900202E0FD2408F582E43402F583E0FEC2
:100AB00074072DF582E43402F583E07C002400FF06
:100AC000EC3EFEEF65327003EE6531600343228039
:100AD000E5226006900206F08038900205E0FEB440
:100AE0000605120CD5802BEEB407051204508022A7
:100AF000900205E0B408051201F18016900205E0AD
:100B0000B4090512098F800A900205E0B40A0312A5
:100B10000BDE020A1B8F1A8E198D188C17851CA7E5
:100B2000AF1AAE19AD18AC1778081207298FF7E580
:100B30001AFF8FFB851BFC75F26E20AF3D75F30528
:100B4000E5A7651C703475F40AE51DB4552C75F5E0
:100B500009AF1AAE19AD18AC177808120729A80406
:100B6000A905AA06AB07AFF7E4FCFDFEC312071800
:100B7000700875F6060000000000E4F5A7228F1447
:100B80008E138D128C118515A7AF14AE13AD12AC58
:100B90001178081207298FF775F2E620AF3C75F33C
:100BA00005E5A76515703375F40AE51DB4552B7579
:100BB000F509AF14AE13AD12AC117808120729A8CD
:100BC00004A905AA06AB07AFF7E4FCFDFEC31207B4
:100BD00018700775F60600000000E4F5A722E490FF
:100BE0000206F0752C0A751D55F515FF7E0EFDFCED
:100BF000120B7EE4F515FF7E0EFDFC120C8C502AC4
:100C0000200130751B5AE4F51C7FFF7E0FFDFC129E
:100C10000B15E4F51B7FFF7E0FFDFC120D94EF64B6
:100C20005A6010900206740380059002067402F068
:100C3000E4F52CE4F51D2253B1F8120DACE4F51BDC
:100C40007FFF7E0FFDFC120D94EF645A7026C201E7
:100C5000751D55120D3850028005120D385005E4EF
:100C6000F51D8024E4F51D758E55438702000000B4
:100C7000000080F0E4F51B7FFF7E0FFDFC120D9459
:100C8000BFA505D2010200A6121000228F148E13F8
:100C90008D128C11D2048515A7E4F516F517AE1642
:100CA000AF17E4FCFDFB7A02F9F8D3120718401FD6
:100CB000E5172514FFE51635138F82F583E493605D
:100CC00004C204800A0517E51770D3051680CFE427
:100CD000F5A7A20422E4900206F0A3E0FFB4490FB6
:100CE000A3E0B4410AA3E0B45005C201D20022EF50
:100CF000B44911900208E0B4530AA3E0B45005D2FD
:100D000001D20022900206740AF0C200227580F817
:100D100075E18F75E9C875908075E27F75EA807519
:100D2000A0E075E33F75EBC075B01975E4E675ECAE
:100D3000194380C043E98022D20312077CEF701967
:100D4000F515FF7E0EFDFC120B7EE4F515FF7E0E01
:100D5000FDFC120C8C92038002C203A2032275C414
:100D600032E4F587759850759D7F759C64759E0477
:100D7000439D80759A0A759BFF2275817F75B20825
:100D8000000000000000000043B20478FFE4F6D841
:100D9000FD020C378F1A8E198D188C17E4851BA74E
:100DA000851A8285198393FFE4F5A722120DB512E7
:100DB0000D0DC20022E4F5A8F5A9F5AA2200000055
:100DC0000000000000000000000000000000000023
:100DD0000000000000000000000000000000000013
:100DE0000000000000000000000000000000000003
:100DF00000000000000000000000000000000000F3
:102344000224E6E86480F8E933E83360110460F0BD
:10235400ED33EC337009E8FCE9FDEAFEEBFF2204FF
:1023640060DED3EB9FEA9EE99DE8C2E78CF0C2F7FA
:1023740095F0400CE8CCF8E9CDF9EACEFAEBCFFBC6
:102384001224B185D0F05804700320D5B3E804704A
:10239400075002B2D50224F092D5EC0460F7E4CCE5
:1023A400C0E0C398F8603B94186008400DD0E0FB8F
:1023B4000224C8E4FBFAC9FC8028E830E406E4C936
:1023C400FBE4CAFCE830E305E4C9CACBFCE85407E3
:1023D4006010F8C3E913F9EA13FAEB13FBEC13FCEE
:1023E400D8F130F52FC3E49CFCEF9BFFEE9AFEED91
:1023F40099FDD0E0FBEF4E4D4C701222DB0302241A
:10240400EDEC2CFCEF33FFEE33FEED33FDED30E766
:10241400EB0224C8EF2BFFEE3AFEED39FDD0E0FBD2
:1024240050130BBB00030224F0ED13FDEE13FEEF7B
:0824340013FFEC13FC0224C8A5
:10243C0075F020800E75F010800575F0087D007E1B
:10244C00007F003392D530D5031226D6EC334010E2
:10245C00EF33FFEE33FEED33FDEC33FCD5F0ED2224
:0E246C00E5F0247EA2D513CC92E7CDCEFF2260
:10247A00EDD2E7CD33EC3392D524814006E4FFFE5A
:10248A00FDFC22FCE4CFCECDCC24E0501174FF80B9
:10249A00EDC3CC13CCCD13CDCE13CECF13CF047056
:0724AA00F030D5DE0226D65A
:1024B100E9D2E7C933E833F892D5EDD2E7CD33EC71
:0724C10033FC5002B2D522EA
:1024C800EC30E7100FBF000C0EBE00080DBD000475
:1024D8000BEB6014A2D5EB13FCED92E7FD2274FF21
:1024E800FCFDFEFF22E480F8A2D574FF13FC7D807A
:0324F800E480EF8E
:1024FB00BB010689828A83E0225002E722BBFE02DF
:09250B00E32289828A83E4932211
:10251400EF8DF0A4A8F0CF8CF0A428CE8DF0A42EDB
:02252400FE2295
:10252600BC000BBE0029EF8DF084FFADF022E4CC99
:10253600F875F008EF2FFFEE33FEEC33FCEE9DEC62
:10254600984005FCEE9DFE0FD5F0E9E4CEFD22EDA8
:10255600F8F5F0EE8420D21CFEADF075F008EF2FF2
:10256600FFED33FD4007985006D5F0F222C398FDE3
:052576000FD5F0EA2280
:10257B00C5F0F8A3E028F0C5F0F8E58215827002EB
:06258B001583E038F02288
:0D259100EF2BFFEE3AFEED39FDEC38FC2299
:0E259E00C3EF9BFFEE9AFEED99FDEC98FC2238
:1025AC00E88FF0A4CC8BF0A42CFCE98EF0A42CFCCE
:1025BC008AF0EDA42CFCEA8EF0A4CDA8F08BF0A44C
:1025CC002DCC3825F0FDE98FF0A42CCD35F0FCEBAB
:1025DC008EF0A4FEA9F0EB8FF0A4CFC5F02ECD3970
:0F25EC00FEE43CFCEAA42DCE35F0FDE43CFC22DD
:1025FB0075F008758200EF2FFFEE33FECD33CDCC97
:10260B0033CCC58233C5829BED9AEC99E582984019
:10261B000CF582EE9BFEED9AFDEC99FC0FD5F0D6F6
:10262B00E4CEFBE4CDFAE4CCF9A88222B800C1B920
:10263B000059BA002DEC8BF084CFCECDFCE5F0CB5E
:10264B00F97818EF2FFFEE33FEED33FDEC33FCEB97
:10265B0033FB10D703994004EB99FB0FD8E5E4F952
:10266B00FA227818EF2FFFEE33FEED33FDEC33FC3F
:10267B00C933C910D7059BE99A4007EC9BFCE99A33
:10268B00F90FD8E0E4C9FAE4CCFB2275F010EF2F78
:10269B00FFEE33FEED33FDCC33CCC833C810D70778
:1026AB009BEC9AE899400AED9BFDEC9AFCE899F8B3
:0E26BB000FD5F0DAE4CDFBE4CCFAE4C8F92246
:106ADC00C2D5E830E70FB2D5E4C39BFBE49AFAE4E5
:106AEC0099F9E498F8EC30E717B2D5126B1212262C
:106AFC0037E4C39BFBE49AFAE499F9E498F8800331
:106B0C0012263730D50DE4C39FFFE49EFEE49DFDB5
:046B1C00E49CFC22D7
:0D26C900EF4BFFEE4AFEED49FDEC48FC2210
:0E26D600C3E49FFFE49EFEE49DFDE49CFC2215
:1026E400EB9FF5F0EA9E42F0E99D42F0EC6480C86D
:0626F40064809845F0220D
:1026FA00EB9FF5F0EA9E42F0E99D42F0E89C45F036
:01270A0022AC
:10270B00E8600FECC313FCED13FDEE13FEEF13FFAC
:03271B00D8F122D0
:10271E00E86010ECA2E713FCED13FDEE13FEEF13D1
:04272E00FFD8F022BE
:10273200E8600FEFC333FFEE33FEED33FDEC33FC05
:03274200D8F122A9
:0C274500E6FC08E6FD08E6FE08E6FF22C0
:0C275100E0FCA3E0FDA3E0FEA3E0FF22FB
:0D275D00E6FB08E6F908E6FA08E6CBF822EC
:0C276A00E0F8A3E0F9A3E0FAA3E0FB22F2
:102776007401FF3395E0FEFDFCA3A3A3E02FFFF059
:10278600E582158270021583E03EFEF0E582158231
:1027960070021583E03DFDF0E58215827002158317
:0527A600E03CFCF02204
:0C27AB00ECF608EDF608EEF608EFF6225A
:0C27B700ECF0A3EDF0A3EEF0A3EFF02295
:1027C300D083D082E493F608740193F608740293DD
:0927D300F608740393F674047314
:1027DC00A8828583F0D083D0821227F31227F312BC
:1027EC0027F31227F3E473E493A3C583C5F0C583E1
:1027FC00C8C582C8F0A3C583C5F0C583C8C582C847
:01280C0022A9
:10280D00D083D082F8E4937012740193700DA3A35A
:10281D0093F8740193F5828883E47374029368606E
:06282D00EFA3A3A380DF6E
:10283300EC8EF0A4CCC5F0CCCDF8EFA4CEC5F02D32
:10284300FDE43CFCE8A42EC8C5F03DFDE43CFCEFF0
:0D285300A4FFE5F028FEE43DFDE43CFC227E
:00000001FF
